:020000040002F8
:10600000588C00207D0C030087740200B7760200D4
:106010005B780200FB7802002B7902000000000090
:10602000000000000000000000000000677A02008D
:10603000A37A020000000000C77A0200AB7B0200D6
:10604000F37D02003F7E020091F102001DEF02008D
:1060500023EF0200B3A8020033B502008D04030051
:1060600061F1020069F1020071F1020013CE020039
:106070006BE60200A1FC020087E8020083F0020048
:1060800093F90200C3F702000FFC0200A50B030006
:106090000B0C0300170C0300ABC00200FF0C030045
:1060A000010D0300030D0300050D0300070D0300A0
:1060B000090D03000B0D03000000000000000000AC
:1060C0000D0D03000F0D0300110D03002DCD020077
:1060D000130D0300150D0300170D03000000000051
:1060E00000000000000000000000000000000000B0
:1060F00000000000000000000000000000000000A0
:10610000000000000000000000000000000000008F
:10611000000000000000000000000000000000007F
:10612000000000000000000000000000000000006F
:10613000000000000000000000000000000000005F
:10614000000000000000000000000000000000004F
:10615000000000000000000000000000000000003F
:10616000000000000000000000000000000000002F
:10617000000000000000000000000000000000001F
:10618000000000000000000000000000000000000F
:1061900000000000000000000000000000000000FF
:1061A00000000000000000000000000000000000EF
:1061B00000000000000000000000000000000000DF
:1061C00000000000000000000000000000000000CF
:1061D00000000000000000000000000000000000BF
:1061E00000000000000000000000000000000000AF
:1061F000000000000000000000000000000000009F
:106200002DE9F84F74A7A2B0D7E90045CDE90045C4
:106210002C9EDFF8307C04918DF843605FF0000124
:106220006FA40D9112944FF0FF3682469046994626
:106230000FE0C3462C461BF8011B0498D0470028EA
:10624000049000F0B2800D98401C641E0D90F2D1B5
:10625000A84498F80000252807D10021079108914B
:1062600009910A910B910C910DE06A463146404626
:1062700001F014F8050001D10D98B5E0D9D501253C
:10628000E6E741F0010118F8010F2028F9D0232892
:106290000CD02B2804D02D2805D0302809D086E03A
:1062A00041F00201EFE741F00401ECE741F00801A1
:1062B000E9E741F01001E6E700200F900AE00F98AF
:1062C000B84205DA00EB800302EB4302303A0F924A
:1062D00008F1010898F80020A2F130000A28EED356
:1062E00098F800002E2818BF0E9629D118F8010F33
:1062F0002A280BD1D9F80000C9F8000008F10108DC
:1063000050F8042BC9F800000E9219E02D280CBF9C
:1063100018F8010B002000220E920BE040B90E9AF3
:10632000BA4205DA02EB820403EB4403303B0E93DE
:1063300008F1010898F80030A3F130020A2AEDD3E1
:10634000ADF84010129898F8001000F0B1FF08B1B5
:1063500018F8010B8DF842009DF84200682804BF30
:1063600098F80010682903D162208DF8420008E0F7
:106370006C2804BF98F800006C2804D171218DF8B6
:10638000421008F1010813A806904A4618F8013B8C
:1063900002A9504600F068F838B913AA02A950467D
:1063A00000F0CAF900287FF554AF30461CE02A28D7
:1063B00082D1D9F80020C9F8002052F8040BC9F89E
:1063C000002000280F9003D540420F9041F00401B7
:1063D00008F1010884E70000000000000000000050
:1063E000686A6C747A4C000023B0BDE8F08F6228B4
:1063F00020D0682811D06A2803D06C2827D07128B3
:1064000025D10868C01D20F007000860D0E90023EE
:1064100008300860194610467047002A0A680A606A
:10642000106803D0121D0A6000B217E0121D0A6046
:1064300080B217E0002A0A680A60106803D0121DB3
:106440000A6040B20AE0121D0A60C0B20AE0002AE7
:106450000A680A60106803D0121D0A60C1177047ED
:10646000121D0A60002170477CB50D4611461C467E
:106470002E69B4F1250200F04D811C3A00F08680AF
:10648000121F022A40F282800E3A00F00781521F4A
:106490005AD0093A7AD0921E16D0521E35D0521ECA
:1064A000022A73D9121F30D0521F00F09A80521E58
:1064B0004AD0521E00F0E480D21E00F0FD80921EF1
:1064C00042D0D21E40D02BE195F83A206C2A09D058
:1064D0006869421C6A610A680A6052F8043B0A60F3
:1064E000335427E10A680A6052F8043B0A6000212D
:1064F000009301914FF0FF322A6329466A4600F06B
:1065000096F9002840F1168101E195F83A00012240
:10651000FFF76DFFC5E900010023994204DA6869BD
:10652000411C69612D210DE0288F810704D5686920
:10653000411C69612B2105E0C00722D56869411C17
:106540006961202131541CE095F83A000022FFF7E0
:106550004EFFC5E9000195F83800010711D5D5E9CE
:1065600000230020834208BF82420AD044F020006A
:10657000782806D1686930213154401C411C69617A
:106580003454214668693044E86083E00868C01DDF
:1065900020F007000860D0E9002308300860C5E952
:1065A0000023D5E90001C80F04D06869411C696166
:1065B0002D210DE0288F810704D56869411C696190
:1065C0002B2105E0C00704D56869411C69612021C1
:1065D000315468693044E8602146284600F032FAB8
:1065E000A8E005F13A02507820B14FF0FF340FF6E1
:1065F000243070E01078622808D0682824D06A28F7
:1066000012D06C282ED071280ED02BE00A680A60B8
:1066100052F8040B0A6020B94FF0FF340FF60C302B
:1066200059E0E96A017085E00A680A6052F8040BD3
:106630000A6020B94FF0FF340FF6F0204BE0EA6A11
:10664000D317C0E9002375E00A680A6052F8040B0A
:106650000A6020B94FF0FF340FF6D0203BE0E96A22
:10666000018067E00A680A6052F8040B0A6020B9EA
:106670004FF0FF340FF6B4202DE0E96A016059E0D5
:106680000A680A6052F8040B0A600021C5E900019B
:10669000EE607821284600F029F94BE06C2285F85D
:1066A0003A200B680B6053F8042B0B6052BB4FF081
:1066B000FF340FF6AC200EE095F83A206C2AF0D0AB
:1066C0000868086050F8044B0860EC603CB94FF073
:1066D000FF340FF6702000F005FE201A76BD2E6BF9
:1066E000002E04D5204600F01DFE044608E0324688
:1066F0000021204600F03EFE002814BF041B344653
:10670000AC6117E0294600F092F8002812D54FF04E
:10671000FF3076BD6869411C69612521315409E06B
:106720006969481C686125227254210002D0411C0D
:1067300069613454002076BD2DE9F0410E460546CE
:10674000716B7069B46A091A306A091AB069091A5A
:10675000706A091AF069091A96F838000C1B41078B
:1067600090460DD4002C0BDD2746B0682021A847A9
:106770000028B06057D0F06A401C7F1EF062F4D150
:10678000736942463146284600F0ACFC00284AD1E5
:10679000376A002F0ADDB0683021A8470028B060B2
:1067A00041D0F06A401C7F1EF062F4D1B369F268F8
:1067B0003146284600F096FCA8BB776A002F09DD19
:1067C000B0683021A847B06068B3F06A401C7F1EF3
:1067D000F062F5D1F068B169F36942183146284694
:1067E00000F080FCF8B9B76A002F09DDB0683021ED
:1067F000A847B060B8B1F06A401C7F1EF062F5D1C6
:1068000096F8380041070BD5002C09DDB06820212F
:10681000A847B06038B1F06A401C641EF062F5D140
:106820000020BDE8F0814FF0FF30BDE8F0812DE998
:10683000F8470D46A3B02F6B002F8146904648BF06
:106840006FF0004700F0C2FD696B40180FF62C1185
:106850008128D1E90023CDE9012328BF4FF0FF3083
:106860003ED20024002F2FDDD8F8001001AA684680
:1068700000F016FD0646002E35D4D8F8000008B901
:10688000761E30D4B7421FDB6869301881280AD3DE
:106890000020686303AA29464846FFF74DFF04001D
:1068A00012D40020686103A8D5F814A032466946C6
:1068B000504400F095FDB244C5F814A058F8040BFC
:1068C000002818BFBF1BCDD12CB903AA29464846C2
:1068D000FFF732FF044614B9002068616863204660
:1068E00024B0BDE8F0874FF0FF34F8E72DE9FC470E
:1068F00007468A463E69BAF16F0F08BF082405D0E3
:106900004AF02001782914BF0A2410243C25D7E935
:106910000023BAF1640F18BFBAF1690F9046994687
:1069200006D100218B4203DAD8F1000869EB49094E
:106930000020814508BF80451FD1386BE8B9082C7D
:106940004CD197F83800010748D530203B2586F810
:106950003B0043E000280ED597F8380000F0140003
:10696000102808D17A6B7869121A386A121A511AEB
:106970000029C8BF3962BDE8F3878DF800A0404602
:1069800049462246E31700F07FFD3032D0B26D1E3B
:106990003A28019504DB9DF80000A0F151018A1806
:1069A0007255404649462246E31700F06DFD804689
:1069B00089460020814508BF804503D0F8687119D9
:1069C0008842DCD3082C09D197F83800010705D597
:1069D000715D302902D06D1E30207055C5F13C012B
:1069E000B9617019F860386B8142B3DA411A3962C3
:1069F0004FF6EF70398F01403987BDE8F3872DE9F5
:106A0000D04306460F4614464FF00008DFF838948E
:106A100012E0E00707D542464B463046394600F0C3
:106A20004BFE06460F464046494642464B4600F05E
:106A300043FE641080468946002CEAD13046394630
:106A4000BDE8D0832DE9F34F054641F020048DB019
:106A5000D5E90089612C02AE09D0286B002848BF17
:106A6000062003D408BF672C01D101202863D5E993
:106A7000002358004015401C0ED119030CD00320F0
:106A8000A8619DF8380061381A2802D20FF2F4612B
:106A900011E00FF2F4610EE058004015401C0FD1D8
:106AA00019030DD10320A8619DF8380061381A2818
:106AB00014D30FF2DC61E868032200F091FCD3E10B
:106AC000194621F00043B3F5801F10460DD2002770
:106AD000BB4208BFBA42019703D111E00FF2AC618B
:106AE000E9E701AA00F0BAFE0AE0DFF8607307EBFD
:106AF0001352DFF85C3301921940DFF85833194321
:106B0000C5E90001612C0ED1E86830210170811CBB
:106B1000E9609DF8381061290CBF78215821417037
:106B20006869801C6861D5E900AB2BF00043002048
:106B30002AF00002834204BF8242002300F05A81FF
:106B4000612C40F0A980286B00284CBF2120401CFC
:106B500000904046009F7F1C49460022002300F021
:106B6000B5FED94601988DF8082038BF89F0004954
:106B7000001F0190002FD0460DF1090040F349811C
:106B800040F2FF71DFF8D0B20C910646404649460C
:106B90000022002300F0B2FE80F03A814800400D50
:106BA00000F11C0210D0002A0EDD0C98824205DB99
:106BB00009F0004040EA0B01002013E0A44808401F
:106BC00040EA025140460DE029F00043002028F041
:106BD0000002834208BF82420FBF40461C2240464B
:106BE00000F0A4FE8046894600F03EFFFF1F002F04
:106BF000044609DD00F056FF02460B464046494672
:106C000000F062FF80468946F01D072104E004F091
:106C10000F0200F8012D2411002C01DD491EF6D5CC
:106C2000491E5CBF002200F8012DF9D5ECE00020E0
:106C3000194602AA0A4400E05B1E12F80149491EE7
:106C40008442F9D00F2804D10DF10900425C521C96
:106C50004254002904D50198001D02AE5B1C01902E
:106C6000591E12D49DF838007218147804F13008B7
:106C70005FFA88F4392CC4BFA0F13A04A044491E3D
:106C800002F80189F1D58DF83800286B002840F111
:106C9000B080591E2963ACE04046494600220023DB
:106CA00000F014FE019938BF89F0004947F297506F
:106CB00041436A4A91FBF2F20192D2F1070204DDEC
:106CC00040464946FFF79BFE0AE0524200206449D5
:106CD000FFF795FE02460B464046494600F066FF28
:106CE0008046662C286BDFF87CB106BF019F0A370F
:106CF00006273F18142FC8BF142730208DF808002E
:106D000089460DF1090000E03046002F34DD0646CB
:106D10004046494601F06EF801460A4606F108036E
:106D200004200A26B2FBF6F606EB860EA2EB4E0214
:106D3000303203F8012C0A22B6FBF2F202EB820E8B
:106D4000A6EB4E063036401E03F8026DE9D1083F2F
:106D5000002F03F10806D7DD084601F05FF8024670
:106D60000B464046494600F0AFFE00225B4600F06D
:106D7000A3FC80468946CBE70DF10901401A0DF1CD
:106D8000090604E00199491E401E0191761C3178E4
:106D90003029F7D0662C02D10199491C03E0652CFB
:106DA0000CBF012100212B6BCB189842B8BF431EAA
:106DB000002B1ED4834204DAF05C3528A8BF3920AA
:106DC00000DA30201946721E02EB010800E05B1E5B
:106DD00018F80199491E8145F9D0392802D1705C13
:106DE000401C7054002904D50198401C16465B1CB9
:106DF0000190019800B200901BB29DF83810324605
:106E0000284600F035F82FE0C61D002F3FF7BEAE34
:106E100030460DF10901401A009903468842C8BF67
:106E20000B46002B0DF109063FF52FAF8342BFF64D
:106E3000FEAE0DF10900C05C07287FF7F8AE0F2009
:106E4000F6E60000CBCCCC0C0000244002FCFFFF97
:106E5000FFFF0F800000E03F0000F07FA0860100F0
:106E60000000F03F84D797410FB0BDE8F08F0000DD
:106E70002DE9F84783B006468A461746984600F043
:106E800011FAB8F1000F406A356B90F8009002DCFF
:106E90004FF00108BFA7BDF930404AF02000662836
:106EA00008BF641C15D0672840F0848014F1040FDB
:106EB000C0F28680AC4280F2838096F83800641C71
:106EC000010702D4A845B8BF454620B22D1A48BFD5
:106ED00000250FFA84FAF068B169BAF1000F25DCD9
:106EE0004A1C30234354002D03DC96F83800010778
:106EF00003D5F06800F80290521C15EB0A0FB8BFDA
:106F00006C4220B2441941424445B8BFA046B26128
:106F100071620FFA88F5F561F068B3692A4639465F
:106F2000184400F05DFA641BB462C4E022B29045DC
:106F3000084417DA4246394600F052FAB069404434
:106F4000B061AAEB0801002D716203DC96F83810DD
:106F50000A0705D5F16801F80090F069401CF0615E
:106F6000B562A8E0394600F03BFAB069002D504404
:106F7000A8EB040803DC96F838100A0703D5F1687B
:106F800001F80090401CB0610FFA88F08542F0686B
:106F9000B369B8BFA8460FFA88F207EB0A01184494
:106FA00000F01EFAB0690FFA88F10844B061681A5F
:106FB000706280E0BAF1610F14D14FF0700A16E0F0
:106FC000A84504DA96F838100A0758BF45466D1EE2
:106FD00048BF0025BAF1670F14BF4FF0450A4FF0C4
:106FE000650A04E0BAF1410F08BF4FF0500AB169D9
:106FF000F368481CB061002D17F8012B5A5403DCCC
:1070000096F838100A071BD5F168431CB36101F8E4
:107010000090002D14DDA8F101080FFA88F08542D8
:10702000F068B8BFA8460FFA88F23946184400F055
:10703000D7F9B0690FFA88F108446D1AB06175622A
:10704000F068B1690844002C80F800A003D42B211B
:107050004170811C03E02D2141706442811C00209D
:107060006A460AE023460A2493FBF4F404EB840501
:10707000A3EB450302F8013B401C24B2002CF1DCD9
:10708000012806DC4AF02002652A04BF302201F8FC
:10709000012B48B9302001F8010B07E0401E1DF814
:1070A0000020303201F8012B0028F7DCF068B269CB
:1070B0001044091AF16196F8380000F01400102805
:1070C0000DD17169B0694118706A4118F0694118B1
:1070D000B06A4118706B8142BCBF411A316204B082
:1070E000BDE8F087F8B505460E4617461C46002059
:1070F00074B117F8011BB068A847B06030B1F06AEE
:10710000401CF0620020641EF3D1F2BD4FF0FF304E
:10711000F2BD00007072696E74665F733A20256E6E
:1071200020646973616C6C6F776564007072696E5E
:1071300074663A2062616420256E20617267756D05
:10714000656E74007072696E74665F733A20626176
:107150006420257320617267756D656E7400000090
:107160007072696E74665F733A2062616420256C88
:107170007320617267756D656E7400000000000019
:10718000000000006E616E004E414E00696E6600A8
:10719000494E46003000F0B4024610689568131856
:1071A000506803EB5004C00721D54D441FE0F0BCEC
:1071B00002F10C00704713F8017B05F8017B491EB2
:1071C000F9D1A0B1B60813F8011B06F00306032E8F
:1071D00008BF13F8016B01EB06214942801C2944CA
:1071E00005D011F8016B05F8016B401EF9D1A342DF
:1071F000DDD013F8016B16F0030104BF13F8011B77
:10720000C91C30090F28DAD113F8010B0F30D6E76B
:10721000FFE741381A288041C00F7047A0F10901EB
:10722000052901D3202801D1012070470020704793
:10723000A0F141011A2938BF203070471A48704721
:1072400030B45368D418042B09DA41B1057804F836
:10725000015B10F8015B15B15B1C491EF3E753603D
:1072600030BC704738B514461D4661B1FFF7E8FFE2
:1072700061686A6B204690476FF00102811A02D064
:10728000491E03D005E06FF0010032BD4FF0FF3022
:1072900032BD0021616032BDDA6B1047024BE1E77D
:1072A000014BF9E70148704720440020E8430020E3
:1072B0000278C9B28A421AB11CBF10F8012FF9E74F
:1072C00018BF00207047B1F5807F02D34FF0FF3028
:1072D00070470170012070470078401E8041C04314
:1072E000C00F704780B500B906A005490B681BB1F7
:1072F00022220021984701E000F09DFD222002BDDE
:107300004C6C0020636F6E73747261696E742068D8
:10731000616E646C65723A20626164206D6573739E
:107320006167650000F10103810704D010F8011BBB
:1073300089B18107FAD10268B2F10131914311F0AC
:10734000803F04BF50F8042FF6E710F8011B11B17D
:1073500010F8011BFBE7C01A70478268521C82605C
:10736000426832B10268531C036011704168491EC3
:1073700041607047C9B2830706D0521E22D310F86D
:10738000013B9942F7D11FE0083A13D302F10402FE
:1073900041EA012141EA014150F8043B121F21BF9B
:1073A0004B40A3F1013C2CEA030C1CF0803FF3D0CE
:1073B000C9B2001F083210F8013B521E28BF91EAE3
:1073C000030FF8D818BF0120401E704780B5FFF7A3
:1073D00035FF006C02BD0268531C036011707047DA
:1073E00062B38B0708D0521E11F8013B00F8013B35
:1073F00000F024808B07F6D1830740F0208000BF87
:10740000103A07D330B4B1E83810103AA0E8381079
:10741000F9D230BC530724BFB1E80810A0E8081027
:1074200044BF51F8043B40F8043BD20724BF31F875
:10743000022B20F8022B44BF0B7803707047121FF9
:1074400017D35B0009D151F8043B20F8023B1B0C19
:10745000121F20F8023BF6D20BE051F8043B00F873
:10746000013B1B0A20F8023B1B0C121F00F8013BDA
:10747000F3D238BF121D521E24BF11F8013B00F891
:10748000013BF8D87047FEE7B3BBD9B1B2F5803FF6
:107490007DD2022A1ED98C46B1FBF2F102FB11C348
:1074A0001B0443EA1043B3FBF2FC02FB1C3380B223
:1074B00040EA0343B3FBF2F002FB103240EA0C4017
:1074C00000237047022A05D98446B0FBF2F002FB84
:1074D00010C270474AB105D100F0010249085FEAC5
:1074E0003000704700220023704700F0A7BC0B005B
:1074F0000200002100207047904271EB030CF6D38C
:10750000B3F5803F2FD2F0B5B3FA83F7B1FA81F427
:10751000A7F10F0E3D1B5340CEF1200602FA0EF2EA
:10752000F3415340B5F10F0746D80F3C2C4441407E
:10753000C4F12006A040F1414140B1FBF3F603FB4A
:107540001611A2FB0645001BA94102D2761E801827
:10755000594180EA010221FA0EF362FA0EF200218B
:107560005A403046F0BD30B4B1FBF3FC03FB1C11B4
:10757000A2FB0C45001BA94103D2ACF1010C801801
:10758000594130BC02460B46604600217047B2F1BB
:10759000807F65D3F0B5B2FA82F7B1FA81F4C7F112
:1075A0000F063D1B22FA06F307F1110EF2412035BA
:1075B0005A40B5F10F07B8D94140C4F12006A040A8
:1075C000F1414140B1FBF3FC03FB1C11A2FB0C4554
:1075D000001BA94103D2BCF1010C801859410F2FA7
:1075E00012D30F3FC90341EA5041B1FBF3F603FB4D
:1075F0001611A2FB0645D4EBC030A94102D2761E7B
:107600008018594146EACC3C07B34140C7F12006F7
:10761000B840F1414140B1FBF3F603FB1611A2FB68
:107620000645001BA94102D2761E8018594180EA06
:10763000010221FA0EF3C7F1200462FA0EF20CFAED
:1076400007F05A402CFA04F13043F0BD80EA010201
:1076500021FA0EF3002162FA0EF260465A40F0BDA4
:107660008C46B1FBF2F102FB11C31B0243EA10632B
:10767000B3FBF2FC02FB1C331B024CEA002043EA82
:107680001063B3FBF2FC02FB1C331B024CEA00202C
:1076900043EA1063B3FBF2FC02FB1C331B024CEA0F
:1076A000002043EA1063B3FBF2FC02FB1C324CEAFD
:1076B000002000237047FEE7B0B581EA030C0CF010
:1076C000004C40F2FF7515EA11541DBF15EA13571F
:1076D000AC42AF4239E0E41923EA455343F4801346
:1076E000C90241F0004141EA505EC7021100A7FB08
:1076F000020200284FF00000EEFB01204FF00001D5
:10770000E3FB072118BF42F0010240180021494164
:10771000E3FB0E01A4F580640F0302D25200404146
:10772000494154F101046CDD470872F1004250F107
:10773000000051EB0451A1F580115CBF41EA0C013E
:10774000B0BD4CEA05510020B0BD05EA1357AC426C
:1077500014BFAF4241E050EA410E1CBF52EA430E53
:1077600002E061460020B0BD24423C441BD15FEAE8
:10777000070EF6D0090302BF01460020AEF1140E39
:10778000B1FA81F7AEEB070401FA07FE0C37C7F137
:10779000200100FA07F7C8404EEA000E23EA4553DD
:1077A00043F48013A2E733F00043B3FA83F704BF36
:1077B000B2FA82FE77440B3FE41BB7F1200E2FBFD5
:1077C00002FA0EF3BB40C7F1200E22FA0EFE38BFBC
:1077D00043EA0E03BA40641C82E750EA410E14BF2C
:1077E00052EA430E6FF000014FF4001717EB430FFE
:1077F0008ABF194617EB410FB5E74CEA0551002047
:10780000B0BDD4F10104B4F120070FDAC4F12007B0
:10781000520828BF42F0010210FA07F501FA07F7F3
:10782000E1BF2A43E0403843E1400FE0352C98DCCB
:10783000C7F1200452EA400220FA07F218BF42F0D2
:10784000010231FA07F0A1400A43002172F100421F
:1078500050F1000051EB0C01B0BDFEE710B514462D
:1078600000F002F8226010BDC1F30A5343B14A0090
:1078700012F5001F28D2A3F2FE32A1EB025170478D
:1078800050EA410C20D001F0004C31EA0C01B1FA71
:1078900081F204BFB0FA80F3D2180B3AB2F12003A0
:1078A0002CBF00FA03F1914041EA0C013EBFC2F146
:1078B000200C20FA0CF319439040524240F2FD3361
:1078C000D21A01EB03517047002270474FF4001C9D
:1078D0001CEB410F94BF1CEB430F09E041EA030C82
:1078E00050EA4C0C52EA0C0C03D2994208BF904269
:1078F000704714BF8B4282427047FEE74FF4001C72
:107900001CEB410F94BF1CEB430F09E041EA030C51
:1079100050EA4C0C52EA0C0C03D28B4208BF824254
:10792000704714BF994290427047FEE7124254D408
:1079300040F2FF7C1CEA11530FD0634531D09B18F5
:1079400063453CBF01EB0251704701F0004141EA41
:107950000C510020AFF30080704750EA410320D063
:1079600001F0004C91EA0C011CD0B1FA81F30B3B01
:107970009A420DD9D21A994051EA0C01C3F1200C58
:1079800020FA0CFC61449840531C40F2FF7CD7E77E
:10799000914041EA0C01C2F1200C20FA0CF319438A
:1079A00090407047B0FA80F31533202BE0D3202AA3
:1079B000EED3203A203B9A4209D9D21A00FA03F1B9
:1079C00041EA0C010020531C40F2FF7CB8E700FAAA
:1079D00002F141EA0C0100207047524240F2FF7C64
:1079E0001CEA11530DD06345DBD0B2EB030C3CBF56
:1079F000A1EB025170470CF1010221EA035141F45D
:107A0000801150EA410CCCD001F0004C352A27DC23
:107A100030B481EA0C01B2F1200309DAC2F120038B
:107A2000044601FA03F5D0402843D1409C400CE0C5
:107A3000C3F12002450020FA03F418BF44F001040A
:107A400021FA03F091400C43002174F1004550F1FC
:107A5000000051EB0C01244230BC7FF47BAF704737
:107A60006146002076E7FEE7C1F30A5340F2FE329A
:107A70009B1A14DDD3F120034FEAE17208DDC9023D
:107A800041EA505141F00040D840801850407047C2
:107A900003F2E13010B1D24382F000407047002081
:107AA0007047FEE7C11768B14840401AB0FA80F24B
:107AB0009040D21CC907C2F5846241EA025202EB2F
:107AC000D02140057047FEE770B44FF0004591EAC1
:107AD000030F40F1B5816B40841A71EB030603D2AA
:107AE000001BB141121973414FF4001C1CEB410FF4
:107AF00034BF7CEB430442E00C0DA4EB1356352E4F
:107B00004FDC45EAC323DB0A45EAC121C912B6F1BD
:107B100020050DDD63FA05F6EB4086EA0305124207
:107B200018BF45F00105C01851F100010CD213E057
:107B300062FA06F5F2405540F3415A40B340F34033
:107B40005A408018594107D349085FEA30005FEA7C
:107B5000350528BF45F0010501F58011420875F192
:107B6000004250F1000041EB04514E0016F5001F99
:107B700070BC38BF70470020090D090570471CEB29
:107B8000410F10D252EA43060BD0BCEB410F05D88F
:107B90000C0DAB43661E342EB6DD02E0AB438018FD
:107BA000594170BC704770BC7047FEE7F0B540F2B9
:107BB000FF7581EA030C0CF0004C15EA11541DBF4F
:107BC00015EA1357AC42AF42E5E0BC41C1F31301E3
:107BD000C3F31303801A994143F4801304D2641E43
:107BE0004000494180185941C90241EA5051B1FB56
:107BF000F3F603FB1611A2FB0675D7EBC020A941D3
:107C000002D2761E80185941C90241EA5051B1FB97
:107C1000F3FE03FB1E11A2FB0E75D7EBC020A9419A
:107C200003D2AEF1010E80185941890241EA905108
:107C3000760546EA8E2EB1FBF3F603FB1611A2FB86
:107C40000675D7EB8020A94102D2761E80185941D3
:107C5000C90241EA50514EEA060EB1FBF3F603FBAE
:107C60001611A2FB0675D7EBC020A94102D2761EE1
:107C700080185941C90241EA5051B1FBF3F703FBA7
:107C80001711A2FB0735D3EBC020A94167F100070C
:107C90000CBF004247F0010766F3D5274FEA1E31BB
:107CA000B80814F5806412DDBD0775F1004250EB91
:107CB0000E5051EB045111F5801F5CBF41EA0C01DD
:107CC000F0BD4CF07F6141F0E0410020F0BDBD0708
:107CD0006D0840EA0E5041F48011D4F10104B4F172
:107CE00020060ADAC4F120060200E04001FA06F399
:107CF000E1401843B24015430EE0342C13DCC6F1CA
:107D0000200445EA40056D0820FA06F2154321FAE1
:107D100006F0A1400D43002175F1004250F1000032
:107D200051EB0C01F0BD00205FEA0C01F0BDCFB9B2
:107D300092185B41B3FA83F704BFB2FA82F6BF1917
:107D40000B3FB7F120062FBF02FA06F3BB40C7F185
:107D5000200622FA06F638BF3343BA401CB1E419B4
:107D6000641E33E77F4231F00041B1FA81F404BF71
:107D7000B0FA80F6A4190B3CB4F120062FBF00FA2C
:107D800006F1A140C4F1200620FA06F638BF3143BF
:107D9000A0403C1B1AE7AC421ABF05EA1357AF429A
:107DA00012E050EA41061CBF52EA4306BFE750EA20
:107DB0004107304661461CBF41EA0551F0BD52EA19
:107DC000430C08BFC143F0BD00204FF4001616EB72
:107DD000410F98BF16EB430F08BF16EB410F24BFAE
:107DE000C14305E016EB430F0CBF61464CEA055159
:107DF000F0BDFEE7400D491840EA81200CD2490D44
:107E0000A1F58061491C40F0004005DBD1F11F0164
:107E100054BFC840C017704700207047014648B1A2
:107E2000B0FA80F18840C91CC1F58461090501EBF5
:107E3000D02140057047012000F0B6B87047FEE73A
:107E4000841A71EB030604D26E40001BB141121973
:107E500073414FF4001C1CEB410F34BF7CEB430615
:107E600082E00C0DA4EB1356362E7BDC012E45EA86
:107E7000C32341DC43EA525312BFD20292025B0891
:107E8000240545EAC12141EA5051D2EBC020994175
:107E900025D407D1B0FA80F610FA06F162D000209E
:107EA000203608E0B1FA81F6B140C6F1200220FA8E
:107EB00002F21143B0404FEAF474B4EB465434F08C
:107EC00001064FEA74040AD8D6F50016760D04F0C0
:107ED0000044F04061FA06F25040F1404840C00AC8
:107EE00040EA415021F0004128BF5FEA500550F1BF
:107EF000000044EBD12135E0DB0A45EAC121C90A83
:107F0000B6F120050EDD42EA0242120CC5F1200650
:107F100003FA06F6EB4042EA06056D42984161F12C
:107F200000010DE062FA06F5F240554063FA06FCE6
:107F300082EA0C02F3405A406D42904161EB03012A
:107F400011F4801F05D1641E620502D06D0040410E
:107F5000494121F48011430875F1004350F10000BC
:107F600041EB045170BC70471CEB410F15D223F05C
:107F7000004352EA43060BD04FEA4C0CBCEB410FD6
:107F800004D80C0D661E342EB7DDEBE7801A99413C
:107F900050EA410608BF0021E4E708BF1CEB430F8D
:107FA00028BF6FF00001DDE72021090326311820EA
:107FB000ABBEF9E700000000000000000000000078
:107FC000F8B50C4615461E4600F03EFE60B128602E
:107FD000012702E045F827007F1C2146002000F021
:107FE00033FE20B1B742F5DB4FF0FF30F2BD38462B
:107FF000F2BD10B50446FFF795F9401E06D4215C8A
:108000000D2912BF0A2900212154F6D0002010BDED
:108010000CB410B5C0B004460A4642AB4FF48071B0
:10802000684600F035FE01461CB9684600F0BEFE09
:1080300008E0012C04D10021684601F03EF901E07E
:108040004FF0FF3040B010BC5DF80CFB012908BFB9
:108050000FF6E00102D011B90FF6E801D8E74FF0B2
:10806000FF3070470A460FF6EC01D1E70A460FF6DB
:108070000411CDE780B518B9BDE8024001F06BBA34
:10808000012908BF4FF0FF3004D0022906D1506803
:1080900001F0F6FBBDE8024001F0DEBAFFE74FF069
:1080A000FF3002BDF8B5054601F028FC0646DFF8B2
:1080B0004C780CE097F8040178B164240FF6803115
:1080C0004FF47A4041F001018847641EF6D101F077
:1080D00015FC801BB0F5FA6FECD301F02DFC0FF608
:1080E000B4012846FFF794FF0020F2BD70B50129C6
:1080F0000446154602D101F03DFC52E0022998A643
:1081000021D1686897A101F055FC18B9204601F00B
:10811000ABFC46E06868314601F04CFC28B92046CB
:1081200001F02CFC012C3CD126E068680178303944
:10813000042936D201F0A4FB042832D2014620469D
:1081400001F050FD2DE003292BD16868314601F084
:1081500031FCA0B9A8681022002101F096FB04466A
:10816000200403D0A1B2002001F0D1FC240C03D0E4
:108170002146012001F0CBFC01F025FD11E0012694
:1081800055F8260001783039042907D201F078FB30
:10819000042803D20146204601F024FD761C022E5D
:1081A000EEDD002070BD7CB5002815462ED10129DA
:1081B000DFF84C670DD13088F189441CA142B8BF6B
:1081C000B489214602B0BDE870400246002001F0AB
:1081D0009BBE02290AD100F042F80446B0898442CD
:1081E000A4BFF089A04237DB2046EAE7032933D158
:1081F00000F035F800F036F8B1898C42A2BFF28960
:10820000A242884228DB8242DBDA25E0022905D13E
:1082100000F025F8BDE8764001F0DCBE032907D167
:1082200000F01DF800F01EF84FF0FF3201460DE09F
:10823000042911D100F013F800F014F80646E8689C
:108240001022002101F021FB02463146204602B0F7
:10825000BDE8704001F063BE4FF0FF3076BD686846
:1082600001F00EBB0446A86801F00ABB38B501292D
:108270000446154602D101F08FFF43E0022924D1C4
:108280006D68B0A100F04BFA58B902F0D0F80028A0
:108290000CBF0FF20C710FF22C712046FFF7B8FEE5
:1082A00030E0287830380A282CD2284601F0E8FA45
:1082B0000546002180B202F07AF800282A4614BF51
:1082C0000FF240710FF2187119E003291AD1686892
:1082D0009DA101F06FFBA8B9A868017830390A297F
:1082E00010D201F0CDFA0546002180B202F07BF8F1
:1082F00000282A460CBF0FF228710FF24871204661
:10830000FFF786FE002032BD1CB5012905D101F022
:1083100043FF01F0BEF9002016BD02291BD15468AD
:108320008AA1204601F046FB10B901F035FFF2E7C3
:108330000FF2F051204601F03DFB0028E9D084A166
:10834000204601F037FB30B901F026FF01F0A1F91A
:1083500001F0AEF9DFE74FF0FF3016BD000000007E
:108360002D6F00002D6400002DE9F0410F46012F14
:10837000A0B040F3DC8014460546666875A100F0A5
:10838000EDF800283AD1042F73A63DD1A06803234D
:108390006A46BDA1FFF714FE032835D1009801F00D
:1083A0006FFAB0F5FA6FA8BFA0F5FA6008900198CF
:1083B00001F066FA401E0790029801F061FA0690FB
:1083C0000323E0686A46B9A1FFF7FAFD03281BD131
:1083D000009801F055FA0590019801F051FA0490C7
:1083E000029801F04DFA039003A802F0FAF8002871
:1083F00040F0A28002F028FA03468AE0ACA100F027
:10840000ADF8D8B9032FABA66ED1A4682046FEF70D
:1084100089FF202868D22021684602F047FA2146C9
:10842000684602F047FA02F0ACFA002859D46B46CD
:10843000324601212846FFF709FE81E00FF2E441B0
:1084400000F08CF830B901F023F80FF218630FF246
:108450000C625FE00FF2146100F080F870B9032F36
:108460000FF2106640D100F0A1F9032800903BD232
:1084700001226946002002F0B2FA31E00FF2FC510D
:1084800000F06CF898B9032F0FF2F8562CD100F0D9
:108490008DF90090401F1A2826D20098DFF8641446
:1084A000C86501226946022002F099FA18E00FF22D
:1084B000DC5100F053F8E0B9052F0FF2D85613D174
:1084C0002069694602F031FB0746E06801F0D8F9FF
:1084D000804600F06BF93B466A46414602F0A9FA35
:1084E000002829D4A36814E031462846FFF7BAFDD6
:1084F00026E00FF2A85100F031F8C0B9032F0FF2B7
:10850000A4560CD1A468204602F0E1FA002813D446
:108510002346324601212846FFF798FD10E0022F3E
:1085200008BFB5A4EFD031462846FFF79BFD4FF0BA
:10853000FF3020B0BDE8F08131462846FFF796FDB8
:108540000020F6E72D6300002D6200006578000032
:10855000616C6C007274630052544300304601F049
:1085600029BA30B50229A5B0044634D155680FF2B6
:108570003C5100F0D4F878BB09A801F0ADF8002117
:108580001DA802F0E9FA15A802F004FBB5A006A99F
:1085900002680A6007A80FF21C51D1E90023C0E964
:1085A00000230DA800F0B6FE02F04EF9034607A81E
:1085B00006A9059004910DA8DFF84C23156815A9AC
:1085C0001DAA029001910092039509AA0FF2EC41B5
:1085D0002046FFF71DFD54E0A3A100F0A0F840B92C
:1085E00002F032F902460FF2F4412046FFF710FD87
:1085F00047E02FA100F093F840B9684601F06CF80D
:1086000000283ED16A460FF2E04137E0B7A100F002
:1086100086F838B90021684602F09EFA6A460FF2E1
:10862000D8412BE00FF2DC4100F079F830B9684610
:1086300002F0B0FA6A460FF2D4411FE00FF2DC41BB
:1086400000F06DF818B9204602F01DFB19E00FF29A
:10865000D44100F064F830B9684600F05BFE6A4629
:108660000FF2C8410AE00FF2344100F058F840B967
:10867000684602F007FA6A460FF2BC412046FFF74F
:10868000C7FC002025B030BD2D00000002F0CCBB9F
:10869000BFF34F8F9D499E480A6802F4E06202438F
:1086A0000A60BFF34F8F00BFFDE700003A000000F3
:1086B000696400004944000080B502F045FC0020D8
:1086C00002BDF8B50229044623D100F025F800B315
:1086D0000FF270410FF27C468A4F00F020F820B96B
:1086E000F87533460FF264420FE00FF2903100F05C
:1086F00016F870B9012000900122694602F06FF966
:108700000120387633460FF27C3201212046FFF7F4
:108710009DFC0020F2BD0000D2F8045083A1284641
:1087200001F048B9F8B50229044624D1FFF7F4FF57
:1087300008B30FF210410FF22446724FFFF7EFFF1C
:1087400028B90120F87533460FF200420FE00FF20E
:108750002C31FFF7E4FF70B9009001226946012037
:1087600002F03DF90020387633460FF2183201212D
:108770002046FFF76BFC0020F2BD70B50429A0B0C5
:10878000144610D1606801F07BF8054600F00EF841
:1087900000EB0536E068694602F0C7F982B2694627
:1087A000304601F063FE002020B070BDA06801F0EB
:1087B00067B880B500F0D5FD002002BD2DE9FC4171
:1087C000054600240FF2A038524E49A70C20604302
:1087D00032584AB1002C12BF414632683946284609
:1087E000FFF716FC641CF1E742A12846FFF710FCD6
:1087F0000020BDE8F6810000000000002DE9F843EC
:108800000446894616469846002500E06D1C0C205B
:10881000684308EB00073968F9B1306801F0CAF81D
:108820000028F3D16CB9387901280FD102F09DFBF3
:10883000BB6832464946002098472EA000F0A5FAB2
:1088400009E07879012808BF02F08FFBBB68324647
:10885000494620469847002001E04FF0FF30BDE830
:10886000F2830000313647007274630038B5044665
:108870008AB00D46012C01BF2878422869784D291D
:1088800004D12946012002F0C3FB2CE02846FFF763
:10889000B0FB0A236A4618A12846FFF791FB05465C
:1088A000002D20DD1B4B00F039F800281BD51A489D
:1088B00003681BB100F032F8002814D50098FEF7C9
:1088C00031FD02280FD300BFA9A12046FFF7A0FB6E
:1088D000009A0FF2F0212046FFF79AFB0FF2F821E1
:1088E0002046FFF795FB0BB030BD000063707500AC
:1088F000257300000D0A00002000000080440020C5
:10890000546B002098420020D44000200CED00E081
:108910000400FA05B0410020386C00206A46294660
:1089200020466BE7746461746100000073646174D5
:10893000610000004F4B202573203A2025730D0A5B
:10894000000000004552524F52202573203A202546
:10895000730D0A004552524F52202573203A204988
:108960006E76616C696420506172616D65746572C8
:108970000D0A00004552524F52202573203A2046DE
:10898000756E6374696F6E204661696C7572650DF2
:108990000A000000646675206F6B0D0A000000007D
:1089A000573235513235364A562C2073756363651C
:1089B000737366756C6C79206572617365642E0DD6
:1089C0000A000000573235513235364A562C206E97
:1089D0006F74206572617365642E0D0A00000000DB
:1089E000536563746F722025642C2073756363650F
:1089F000737366756C6C79206572617365642E0D96
:108A00000A000000536563746F722025642C206E89
:108A10006F74206572617365642E0D0A000000009A
:108A2000426C6F636B2025642C20737563636573E0
:108A30007366756C6C79206572617365642E0D0ABE
:108A400000000000426C6F636B2025642C206E6F69
:108A500074206572617365642E0D0A00544441549C
:108A60004100000053617665640000006D6F64652D
:108A7000000000004D4F4445000000007061757318
:108A8000650000005041555345000000646366676F
:108A90000000000044434647000000006E616D6521
:108AA000000000004E414D4500000000696E666FF9
:108AB000000000003230303044505300494E464FE1
:108AC0002C25732C25732C25732C25732C25732CA6
:108AD00025732C25732C257300000000525443206D
:108AE0003A2025730D0A00004445565F4944203A58
:108AF0002025730D0A000000435055203A202573AD
:108B00000D0A00006370755F696400004350555F93
:108B10004944203A2025730D0A0000006661756CF7
:108B2000740000006164647200000000414444521B
:108B3000203A2025730D0A004E414D45203A20254C
:108B4000730D0A0074726967676572005452494771
:108B500047455200454E41424C454400444953412B
:108B6000424C4544000000002C202573000000000A
:108B70000D0A2D2D2D2D2D2D2D2D2D2D2D2D2D2D68
:108B80002D2D2D2D2D2D2D2D2D2D2D2D2D2D2D2D15
:108B90002D2D2D2D2D2D2D2D2D2D2D2D2D2D2D2D05
:108BA0002D2D2D2D2D2D2D2D2D2D2D2D2D2D2D2DF5
:108BB0002D2D2D2D2D2D2D2D2D2D2D2D2D2D2D2DE5
:108BC0000D0A00002573203A206E6F7420646566DC
:108BD000696E65642E0D0A00232323232323232398
:108BE0002323232323232323232323232323232355
:108BF0002323232323232323232323232323232345
:108C00002323232323232323232323232323232334
:108C10002323232323232323232323232323232324
:108C20002323232323230D0A00000000000000005B
:108C30000000000000000000000000000000000034
:108C40000338FDD87047000038B504000D4609D040
:108C5000204602F0EFF90444207848B90B4A00217D
:108C6000116032BD09480468002CF1D1002032BDEA
:108C70002946204602F0EFF92118087810B10022A9
:108C800001F8012B2046014A116032BD486C0020DA
:108C900008B584B00023039300290EBF019301900F
:108CA000491E0291009301A904AB0748784418308B
:108CB000FDF7A6FA019909B100220A70002858BFF1
:108CC000039805B000BD00BF93E6FFFF01780029BF
:108CD00000D070471CB5684602F0A5FA69480188C3
:108CE0009DF80020491C01807F2A674901F5A16495
:108CF000608802D1C8B1401E16E00D2A18BF0A2AAA
:108D000007D100220A540120207002F001FB00204C
:108D10000AE0B0F5807FA4BF0020608062889DF8E3
:108D2000000088546088401C608013BD38B58AB04C
:108D30000DF1100057A1544C1822FEF761FB4FF4BF
:108D40008070019004F20C614FF4806002910390F6
:108D500004F20C55009507234C4A694604A802F01A
:108D600003FA04F5A06100220A720A604A6018B191
:108D700002F008FB4FF0FF300BB030BD42487047A7
:108D80004149002081F8080570470EB400B5C0B015
:108D9000024641AB4FF480716846FFF779FF014608
:108DA000684600F003F840B05DF810FBF8B50546E2
:108DB0000E46374CEFF3058109B33348002700F521
:108DC000A06106E015F807C002447F1C82F800C1CC
:108DD0004B60B7420CDA4A68D1F800C0531CB3F5B7
:108DE000806FA8BF00236345ECD16068401C6060C1
:108DF000002FC4BF062002F08BFA3846F2BD21785E
:108E0000012903D16068401C606010E001212170DD
:108E1000002700E07F1CB7420CDAE85D02F0B8FAE8
:108E20000028F7D06068401C0021606021704FF07E
:108E3000FF30F2BD002100282170F8D13046F2BD8C
:108E400038B5114C04F5A06507E02868401C28607F
:108E5000B0F5806FA4BF0020286028686968884248
:108E60000DD0204490F8000102F092FA0028ECD0D6
:108E700007484168491C41604FF0FF3032BD002077
:108E800032BD0000546C002004570020CD8C02003D
:108E9000106C00201A0000001C000000FFFFFFFF04
:108EA000FFFFFFFF0000000000E0D701000000000E
:108EB00010B5040008D00FF2C8514FF47A4041F0C9
:108EC00001018847641EF6D110BD00B5C1B0112163
:108ED0008DF800100246BDA101A802F073FA01A8A6
:108EE000FEF720FA1F28C8BF1F2082B201A96846DA
:108EF0007CDF08B14FF0FF3041B000BDE0B5FFF7B7
:108F0000E4FF0021CDE900110620ADF80410ADF812
:108F10000000ADF802004FF4C871ADF806106846C5
:108F20007ADF08B102F06EFA07BD02F06BBA7CB5C9
:108F30000546287858BBAA8A1646012E27DDDFF899
:108F4000584429692046FEF74BFA0020A05504F545
:108F500080720120A98A50711160107990B920782F
:108F600001231371422804BF62784D2A04D10FF205
:108F70005840FFF70AFF05E00A4621460FF260401D
:108F8000FFF703FFBDE87640022002F0C1B973BDD0
:108F90001CB5DFF80804DFF80844019001A904F1CA
:108FA000280002F040FA08B102F02CFADFF8F403CE
:108FB0000090694604F10C0002F064FB08B102F075
:108FC00021FA13BD007840B9DFF8D42310883B2183
:108FD00076DF002818BF02F015BA704702F012BA07
:108FE00000B587B01C21684601F060FC00200090AD
:108FF0004FF4A0314FF4F0200290019100200321A2
:10900000ADF80E008DF810008DF80C10DFF8980305
:10901000DFF8981305900691684602F034FC08B119
:1090200002F0F0F907B000BD704730B50446ABB0B0
:1090300021460FF2C430DFF86853FFF7A6FE6C60DC
:10904000AC21684601F032FC02208DF800000021BE
:109050008DF8021006208DF803000121ADF84C10A8
:1090600005F134008DF87C10149000211FA80161D7
:10907000C460DFF83C13DFF83C4381622046694658
:1090800002F0E7FC08B102F0BDF90121204602F030
:10909000DDFC2BB030BD80B50321DFF8180302F0F2
:1090A0004DFD18B1BDE8024002F0ACB901BD38B5C4
:1090B000DFF8EC5204462188288810290CD01129A9
:1090C0001AD013293AD021292FD03B2940D0522938
:1090D00039D056293CD031BD0FF23030FFF755FE64
:1090E000A188298005F1280002F0AFF908B102F04B
:1090F00089F902F069FE31BD4FF6FF7028800FF24A
:109100002030FFF742FEAC4801686868A96040283B
:109110001CBF4020FFF789FF02F062FE9E4900203D
:1091200081F80401FFF7B7FF31BD0FF25C30018811
:10913000ADF800106946A0888FDF0CE00023002204
:1091400085217FDF07E0002300220021B1DF02E05C
:10915000A088132176DF08B102F054F931BD80B543
:1091600002F01AFF08B102F04DF9002000906946A4
:10917000012002F0AFFF08B102F044F9684603F0A5
:1091800004F808B102F03EF901BD85484B88028819
:109190009A4202BF0A8840F677239A4202D1898810
:1091A000CA1E4280704710B5844C8549204603F0A2
:1091B00045F808B102F026F9F721204603F054F8EB
:1091C00018B1BDE8104002F01DB910BD25730000B4
:1091D00038B50446704D05F23C521021C02003F012
:1091E00009F908B102F00EF9FFF7B9FF2046FFF7C1
:1091F00085FEFFF7D8FFFFF7CBFE4020FFF715FFF6
:10920000FFF7EEFE0A20FFF753FE05F582700021FE
:1092100001808170FFF73FFF02F0E2FD002032BDC8
:109220005D4870475C48D0F8000170475A490020FB
:1092300081F805017047F0B504466248154602788A
:10924000C1B00AB908202BE08078012811D14FF471
:10925000807301AA204603F0EFF8002807DD01AA79
:109260000A211154401C01ACADF8000003E00020BD
:109270001AE0ADF800100026012D494F08D100F08A
:1092800015F868B9BDF800000EE00120FFF710FEE8
:1092900000F00CF81328F4D1761C332EF5D30D20F2
:1092A00002F070F84FF0FF3041B0F0BD3B886A46E5
:1092B000214607F10C0002F04EBA38B504460D46BF
:1092C000FEF730F881B22A462046BDE83840B2E7C2
:1092D0000CB40A4610B53049044691F80401C0B0F8
:1092E00028B9082002F04EF84FF0FF300EE042ABF4
:1092F0004FF480716846FFF7CBFC0028D8BF0020F0
:1093000004DD81B222466846FFF795FF40B010BCED
:109310005DF80CFB10B5044686B00020207004A850
:109320006DDF010006D000BF43A0FFF72EFD4FF018
:10933000FF3014E09DF811009DF812100390029187
:109340009DF813009DF81410019000919DF81530C0
:109350009DF8162040A1204602F034F8002006B007
:1093600010BD0F4800884FF6FF7290421CBF1321BA
:1093700076DF7047084890F80411012900D1704742
:1093800080B590F85C0174DF4FF44870FFF74DFE34
:10939000BDE801407FE60000804400202B8F0200E2
:1093A000E44000202F8F0200C58F0200DD8F0200F5
:1093B000299002008845002098420020946B0020EC
:1093C0008B91020084450020424C455F4D45534738
:1093D000203A20424D20282564290D0A0000000073
:1093E000424C455F4D455347203A202573202825A0
:1093F00064290D0A000000004144565F494E54455F
:109400005256414C203A2025640D0A00424C453EFC
:109410003E20636F6E6E65637465642E0D0A0000F6
:10942000424C453E3E20646973636F6E6E656374A3
:1094300065642E0D0A00000073645F626C655F67EF
:1094400061705F616464725F6765742829202D3ED6
:109450002025640D0A000000253032583A253032AC
:10946000583A253032583A253032583A2530325859
:109470003A253032580000000000000000000000D3
:109480000338FDD870470000000000000000000015
:109490002DE9F0470446C0B000F005F9002807D5D3
:1094A0004FF480518DA0FFF770FC4FF0FF3044E087
:1094B00003F063F803F0B6F8009001F0D5F80190DE
:1094C0004FF0FF30039002940424DFF884A1614E32
:1094D000DAF800000FF22829876800204FF480583E
:1094E00030609625DAF8000000EB87006B460169D2
:1094F000102203EB8400FDF773FF7F1C962F28BF1B
:109500000027241D402C0BD300F01AF800F01DF8A2
:1095100003F033F8306808EB8408401C0024306006
:109520006D1EDFD144B100F00BF800F00EF803F02F
:1095300024F83068401C3060002040B0BDE8F0875F
:10954000A2006946404603F036B80346A2004146F1
:109550004846FFF71ABC2DE9F04F83463D480168A5
:109560000A29C5B04FF4805938BF4FF0FF3043D3BC
:1095700000240FF2D0180FF2A81A05AE4FF4807233
:1095800005A9484603F003F809F5807964B97068C5
:1095900001F054F90346B068059A009051465846C8
:1095A000FEF736FD012505E0092C02D1002507272D
:1095B0001CE00025102719E006EB05106D1CB0F922
:1095C0000C100491B0F90A100391B0F90A1002913D
:1095D000B0F906100191B0F904100091B0F9023011
:1095E000B0F9002041465846FEF712FDBD42E3DBCC
:1095F000641C0A2CC2DB002045B0BDE8F08F154981
:1096000018B50A680A2AA1B01BD344F25441C30119
:10961000ADF80010ADF8020003F580531228B9BF71
:10962000802284247022742401A9184602F0AFFF1E
:10963000002806D4012221466846FFF7FCFD0028D9
:1096400002D54FF0FF3000E0002022B010BD000036
:10965000FC420020D040002038B5002811D500255C
:109660002846FFF7CCFF32243DA14FF47A4041F069
:1096700001018847641EF7D16D1C132DF0DB00201B
:1096800032BD132802D34FF0FF3032BDBDE8324067
:10969000B5E780B500F007F8002802D54FF48051F7
:1096A00012E0002002BD01214FF4805002F09EBF65
:1096B00080B50121002002F099FF002801D500218A
:1096C00002E0002002BD000004A0FFF75EFB4FF0A7
:1096D000FF3002BD01F055B901F012B97379735F23
:1096E000666C6173685F65726173652825642C2000
:1096F00031292C206661696C65642E0D0A0000001A
:109700007379735F666C6173685F777269746528DB
:1097100025642C20256429202D3E2025640D0A0077
:10972000426174746572793D25640D0A54696D65F2
:109730003D25730D0A547269676765723D25640D96
:109740000A00000025642C25642C25642C25642C3B
:1097500025642C25642C25640D0A000000000000FF
:109760000338FDD8704700002DE9FC4F83B00E464A
:1097700017460BB100221A608046444600E0641C84
:10978000207802F06BFF0028F9D120782D2816BF31
:109790002B2814F801BB4FF02B0B002F019603D49C
:1097A000012F01D0252F04DB002E47D0C6F8008002
:1097B00044E0002F0ADD102F04BF2078302802BFBC
:1097C000617841F0200178290ED10AE02078302814
:1097D00018BF0A2708D1607840F02000782802D10D
:1097E0001027A41C00E00827029400E0641C2078E5
:1097F0003028FBD04FF0000925A02646CA468DF838
:10980000000007E09DF80050451BCA46EDB207FB7B
:109810000959641C207802F02BFF00BF1CA30146ED
:109820003A461846FDF7A6FD0028EBD10299A14261
:10983000484605D1019808B1C0F8008000201CE01E
:109840001DA1A61BC95D761A002E0FD405DC451B91
:1098500003D3B5FBF7F1514508D0AFF3008004986E
:1098600008B1012101604FF0FF3003E0BBF12D0F83
:1098700008BF4042019901B10C6005B0BDE8F08F0E
:10988000FFE700230A2200216EE700BF00236BE7F9
:109890003031323334353637383961626364656666
:1098A0006768696A6B6C6D6E6F70717273747576D0
:1098B0007778797A0000000000002115110E0D0C58
:1098C0000B0B0A0A09090909090808080808080809
:1098D000070707070707070707070707070000002D
:1098E0001149124A0120086001211148416081603C
:1098F0002021116001220260002070470D4800689D
:109900007047884201D3401A7047C1F180714018F6
:10991000704708490968814201D3081A7047C0F1AD
:1099200080700818704700000800004008150140CA
:10993000001001400415014011DF0849B120086002
:10994000BFF34F8F064907480A6802F4E0620243FA
:109950000A60BFF34F8F00BFFDE700BF1C0500404A
:109960000CED00E00400FA050B4601460822104801
:1099700002F0AFBE0E49498800F034B938B50C4D3D
:1099800004466888411E8941C90F204600F02AF923
:10999000002802D54FF0FF3032BD6988204600F024
:1099A00021F90546012C08BF00F00DF9284632BD0B
:1099B000806B002081EA00039B0717D1820707D044
:1099C00010F8012B11F8013BBAB19A42F6D014E01D
:1099D00002680B689A42A2F1013301BF934313F06E
:1099E000803F50F8042F51F8043FF3D010F8012BBA
:1099F00011F8013B0AB19A42F8D0D01A7047000022
:109A000028B10FF25C21800141F001010847704745
:109A100010B5044600F028FE20600020207102F0FE
:109A200004FE6071DFF8E8010188E18010BD462086
:109A3000E6E71CB504466846FFF7EAFF234608221E
:109A40006946744802F045FE16BD1CB504466846DA
:109A5000FFF7DEFF02218DF80410ADF8064000216B
:109A60006846FFF781FF16BD38B56A4D0446688821
:109A700002280CBF03210221204600F0B3F8002881
:109A800002D54FF0FF3032BD69882046BDE8344032
:109A9000A8E0000070B5064686B00C461546680979
:109AA0000002EB0000EB043003F0F803082204A9E5
:109AB000181800F01CFCFFF7BAFF9DF9140010F114
:109AC000010F21D0022804980CD100F0B7FEBDF898
:109AD00016109DF815200291019200902B46224607
:109AE0004DA10EE000F0AAFEBDF816109DF815205D
:109AF0000190039102922B469DF914004FA1009012
:109B000022463046FEF784FA002006B070BD2DE9EB
:109B1000F84FA2B08846060345F244410001ADF873
:109B200004104FF0010A4FF0FF3B002500904FF664
:109B3000FF7901AF18EA0A0F4FEA4B0B36D00098B5
:109B400028187880802202A9304600F0D0FB002837
:109B500036D40A244FF47A70FFF752FF641EF9D10D
:109B6000002101A800EBC10082884A4504BFC088DB
:109B7000484502D0491C1029F3DB102903DA788804
:109B800040F44040788018EA0B0F03D1788840F405
:109B900000407880C900091D002289B201A8FFF7A2
:109BA0004AFB00280CD47888010405D480366D1C4B
:109BB000202D4FEA4A0ABDDB002023B0BDE8F08F1C
:109BC0004FF0FF30F9E780B545F244404FF6FF71A2
:109BD000ADF80000ADF80210002204216846FFF73E
:109BE0002AFB02BD38B50C4658B900252A46214645
:109BF0000020FFF74FFF6D1CB5F5007FF6D3002066
:109C000032BD2046BDE834404FF6FF717FE70000CB
:109C1000546B00206C6B00202564253033642020B9
:109C200074696D655B545D203A20202573202533CF
:109C3000642020543A25640D0A0000002564253074
:109C40003364202074696D655B25645D203A2020B3
:109C50002573202533642020423A25640D0A000034
:109C60000338FDD87047000000000000000000002D
:109C700028B10FF21C51800141F0010108477047E3
:109C800010B5040005D04FF47A70FFF7F1FF641EA1
:109C9000F9D110BD38B501469A4D1022284602F080
:109CA000A6FD040004BF288900280BD1A98A2888B2
:109CB000814207D002F06DFE29880FF2C430A982DC
:109CC000FFF763F8204632BD000000002DE9F04F99
:109CD0008C4B8BB09C89A142A1BF0A92DB890A9A66
:109CE000934205DA072001F04DFB4FF0FF3082E090
:109CF0008146002500248A4601E00AF1010A8148D4
:109D0000C189491C8A4508BFB0F80CA00FF2843104
:109D100052464846FEF77CF900260027300300EB48
:109D20000A404FF0000B00EB0728102206A908EBB1
:109D30000B1000F0DCFABDF9182012F1010F04BF7E
:109D4000BDF91A0010F1010F23D1BDF91C0010F16B
:109D5000010F04BFBDF91E0010F1010F19D1BDF9AB
:109D6000200010F1010F01BFBDF9220010F1010F19
:109D7000BDF9240010F1010F0BD1641C022C25DD6C
:109D800011271026002D27DDC5A14846FEF740F912
:109D900022E0BDF92430BDF926000FF258310493BA
:109DA0000590002CBDF92030BDF9220002930390EC
:109DB000C8BF0024BDF91C30BDF91E0000930190FE
:109DC0004846BDF91A30FEF723F96D1C0BF1010B63
:109DD000BBF1100FA9DB7F1C102F9FDB761C102E10
:109DE0009BDB0A98824588D14FEA0502CBA1484601
:109DF000FEF70EF900200BB0BDE8F08F38B5FFF785
:109E00007DFD044640F6B83502E0FFF777FD0446D5
:109E10002046FFF77EFDA8420BD201F095FA002103
:109E2000012002F024FE0128EFD00120FFF728FFD7
:109E3000EEE731BD2DE9FE4F324DA8890F4687422E
:109E4000A2BF0292E989914206DA072001F09AFA4C
:109E50004FF0FF304EE07F1CE989B8B2491C8842C0
:109E6000C4A008BFAF891FFA87F94946FEF78DFFE6
:109E70000026ADF80070B046ADF80280002400E086
:109E800014B902F073FE03E0032C08BF02F070FE69
:109E9000ADF804404FF0000A01F056FA002101200D
:109EA00002F0E5FD0AEBCA00ADF80600002301222E
:109EB000B1B2684602F095FD83464620FFF7D8FE12
:109EC000761CBBF1840F17D30AF1010ABAF1010F16
:109ED000E2DD641CA4B2102CD2DB08F101081FFAE9
:109EE00088F01028C8DB02988145B4D1002002F028
:109EF000EBFD0020BDE8FE8FFFF780FF1024A04699
:109F0000E7E70000546B0020002808BFFFF7DEBE23
:109F1000012808BFFFF78EBF4FF0FF3070472DE9D3
:109F2000F845A2B00C4644F25341ADF800109046FB
:109F30006101ADF80410ADF80200210301270025EE
:109F4000002601EB004A18EA070F24D006EBD67072
:109F50004010F3010AEB002003F0800380220DF192
:109F60000601181800F0C3F9BDF8060080B100F032
:109F700078F803DB0F2C08BF1F2E02D100F063F826
:109F8000012500F067F80A20FFF77AFE65B902E0C4
:109F90004620FFF76DFEBDF804007F00761C401CD4
:109FA0001F2EADF80400CEDD85B9BDF8020040F4E7
:109FB0000040ADF802000022BDF8040040F400406B
:109FC000ADF8040006216846FFF735F9002023B0FC
:109FD000BDE8F085F8B5A2B0044644F25340ADF8B0
:109FE0000000ADF802400020ADF804000026240473
:109FF000002740F2FF1580220DF10601204600F0F7
:10A0000076F9BDF8060078B100F02BF801DBAF421D
:10A0100002D100F018F8012600F01CF80A20FFF722
:10A020002FFE30000CD102E04620FFF721FEBDF8E4
:10A03000040080347F1C401CAF42ADF80400DADD20
:10A04000002023B0F0BDBDF8021041F40041ADF88E
:10A05000021070470001801D81B200226846FFF7A0
:10A06000EAB800204FF6FF730DF106010201895A8C
:10A07000994202D0401C0828F6DB082870470000EF
:10A0800073646174615F626C6F636B203A20256456
:10A090000D0A0000626C6F636B2025640D0A0000DE
:10A0A00053545245414D5F454E44212121212121E8
:10A0B0002121212121212121212121212121212190
:10A0C0002121212121212121212121212121212180
:10A0D0002121212121212121212121212121212170
:10A0E0002121212121212121212121212121210D74
:10A0F0000A000000253032642C253032642C2530D3
:10A1000032642C253032642C253032642C253032D8
:10A11000642C253032642C25640D0A00454E442100
:10A12000212121212121212121212121212121211F
:10A13000212121212121212121212121212121210F
:10A1400021212121212121212121212121212121FF
:10A1500021212121212121212121212121212121EF
:10A1600021212121212121212121282564290D0AB4
:10A170000000000073656E7420626C6F636B203AA0
:10A180002025640D0A00000000000000000000000F
:10A190000338FDD87047000038B5002408A5002119
:10A1A000A0B200F004F921462846FEF7EEFD641C3B
:10A1B0000E2CF4DB07A0BDE83240FEF7E6BD000040
:10A1C00045726173652025645F736563746F720DFA
:10A1D0000A000000457261736520646F6E650D0AA8
:10A1E000000000000000000000000000000000006F
:10A1F00028B10FF22C31800141F00101084770476E
:10A200001FB5069C009101920293039400226946B7
:10A21000001D02F024FD04B010BDF8B511F1010FCE
:10A220000CBF531C531D092B01DB0720ADE0C3F10C
:10A230000805DFF8D442261DEFB26D1CF05511F170
:10A24000010F0FD0EFB2080EF0556D1CEFB2080CE5
:10A25000F0556D1CEFB2080AF0556D1C201DEEB2D2
:10A260006D1C8155100006D0211DEEB200206D1C22
:10A270008855521EF8D11846F2BD1CB50A46002179
:10A2800000911218DFF880424042204400F10C0196
:10A290000023D2B2DFF87402FFF7B2FF18B101F069
:10A2A00071F84FF0FF3016BDF8B51D461446024652
:10A2B00008182918C9B2DFF8506200915242B71845
:10A2C000C2B207F1940307F10C01DFF84002FFF777
:10A2D00097FF00B159E02CB12A4606F194012046BF
:10A2E000FDF77EF80020F2BD0021C0B2DCE770B5BA
:10A2F0000C46154640F201118D42064605DA06F07D
:10A30000FF01C1F58071914201D207200AE0802D42
:10A3100012DD00F018F8802322460021C0B2FFF7BA
:10A32000C3FF20B101F02EF84FF0FF3070BD00F0F8
:10A3300079F88034803D803600F005F8EBB2224693
:10A34000BDE87040D0E700223146132065E76E4932
:10A350000620FFE7C872002101208EE70A4680B57B
:10A36000411E03290BD26A4B67491844012310F898
:10A37000010CC8720021BDE80050012094E70720BD
:10A3800001F000F84FF0FF3002BD00F0FBFF4FF08E
:10A39000FF30F2BD80B569460120FFF7DFFF0028DE
:10A3A00006BF9DF8000010F00100012002BD38B585
:10A3B0000446B4F5005F0D46A8BF07200CDAFFF78E
:10A3C000C6FF48B900F02EF8002221032120FFF734
:10A3D00024FF00F029F800B100E01AE000F0D2FFFD
:10A3E0004FF0FF3032BD38B50446B4F5007F0D465E
:10A3F000A8BF07200CDAFFF7AAFF48B900F012F84F
:10A4000000222104DC20FFF708FF00F00DF800B166
:10A41000E4E72DB900F006F8FFF7BCFF0128F9D0FA
:10A42000002032BD4620E3E60021C0B225E710B58A
:10A430000446FFF78CFF50B9FFF7F4FF00224FF0FE
:10A44000FF31C720FFF7E9FEFFF7EEFF00B108E09C
:10A450002CB9FFF7E7FFFFF79DFF0128F9D0002097
:10A4600010BD00F08FFF4FF0FF3010BD2DE9F0411F
:10A470000646154640F2011085420C4605DA06F004
:10A48000FF00C0F58070A84201D207202CE0FFF742
:10A490005EFF002828D1FFF7C5FF802DDFF8688018
:10A4A00017DD00F02CF80746802200F023F8802109
:10A4B000F8B2FFF7E2FEB8B9FFF7B4FFFFF76AFFA3
:10A4C0000028F9D1FFF743FFFFF7ACFF8034803D50
:10A4D000803600F014F80646AAB200F00BF8E9B294
:10A4E000F0B2FFF7CAFE18B100F04CFF4FF0FF309A
:10A4F000BDE8F081214608F10C00FCF771BF002295
:10A500003146122089E6000094660020884200202F
:10A51000A443002000000000000000000000000034
:10A520000338FDD870470000002101E0491C0A38BB
:10A530000A28FBDA40EA0110C0B2704701090A227A
:10A5400000F00F0012FB0100704730B585B00446E3
:10A55000002008218DF80800019103AD009500F05E
:10A560007AF802F014FC60B100202061182101206B
:10A57000E06061610020A060606020604FF0FF300B
:10A580002DE0687800F07F00FFF7D8FF20609DF88D
:10A590000E0000F07F00FFF7D1FF60609DF80F0014
:10A5A00000F03F00FFF7CAFFA060287900F03F00ED
:10A5B000FFF7C4FFE0609DF81100FFF7BFFF00F058
:10A5C0000700A0619DF8120000F01F00FFF7B6FF22
:10A5D000401E2061E879FFF7B1FF6061002005B0FF
:10A5E00030BD30B585B0044600208DF808008DF8E8
:10A5F0000C0003AD2068FFF797FF68706068FFF7F5
:10A6000093FF8DF80E00A068FFF78EFF8DF80F0006
:10A61000E068FFF789FF2871A069FFF785FF8DF8D3
:10A6200011002069401CFFF77FFF8DF81200606960
:10A63000FFF77AFF8DF8130003A90820019000911D
:10A6400000F009F802F0B8FB18B100F09BFE4FF0E3
:10A65000FF3005B030BD012302AA512101487047E7
:10A66000000000001443002000B58BB06846FFF7DF
:10A670006CFF684600F002F80BB000BDF8B5054667
:10A680008CB02F69EE686C6974A168463022FCF7C3
:10A69000B7FE04F5FA64611E40F26D13880803FBEF
:10A6A00001036420B1FBF0F29A1A4FF4C873B1FBB6
:10A6B000F3F15DF827008A188218012F11D914F0E0
:10A6C000030F06D16420B4FBF0F0642101FB1040BD
:10A6D00030B9B4FBF3F34FF4C87000FB134404B972
:10A6E000521CB61851496C68AB688E193C204FF467
:10A6F0006161444328684E4A01FB0343C31802FBCF
:10A70000063630460DB0F0BD10F0030F14D16421B1
:10A71000B0FBF1F1642202FB110159B94FF4C87387
:10A72000B0FBF3F34FF4C87101FB1300401E8041EE
:10A73000C00F704701207047002070472DE9F0419D
:10A740003B493C4EB0FBF1F501FB15003C22B0FB50
:10A75000F2F23C2101FB1202B2614FF46161B0FBE5
:10A76000F1F201FB12003C23B0FBF3F0F061072192
:10A77000281DB0FBF1F1C1EBC101401A3262306318
:10A7800040F2B27740F26D144FF4B77809E0854299
:10A7900025D300F033F8012814BF204640462D1A77
:10A7A0007F1C00F02BF801280CBF40462046EEE746
:10A7B000B46A3044005D854218D300F01FF80128C8
:10A7C00014BF00200C203044005D641C2D1AB462BC
:10A7D00000F014F801280CBF0C200020E8E7A7F5D2
:10A7E000FA60F06275630020B062F1E700206D1C32
:10A7F000B063756206F11800BDE8F081384683E762
:10A800001FB501680C4C0391416802918168019168
:10A81000C1680091036942691CA15B1C02F5FA62E0
:10A82000204600F0CFFD204604B010BDC506F5FF60
:10A83000805101008C400020186B002080B5FFF78C
:10A840007DFFBDE80240DBE700B58BB06846FFF74F
:10A850007CFE6846FFF7D4FF0BB000BD000000008F
:10A860001F0000003B0000005A00000078000000BC
:10A8700097000000B5000000D4000000F3000000C5
:10A8800011010000300100004E0100002530346449
:10A890002D253032642D2530326420253032643A43
:10A8A000253032643A25303264000000002202F084
:10A8B000B1BAFEE75FEA000C80EA01039B0715D1FD
:10A8C000830706D011F8013B00F8013BB3B18307C1
:10A8D000F8D10A68B2F1013323EA020313F0803F92
:10A8E00002BF40F8042B51F8042FF3E711F8013BA5
:10A8F00000F8013B13B111F8013BF9E760467047DE
:10A9000010B50446002020702022214601F03FFEB1
:10A91000002800D5D8E02078FF2804BF6178FF29FF
:10A920000BD1A078FF2804BFE178FF2905D163A0EF
:10A9300001682160052000F025FD002010BD80B5D4
:10A9400001464FF40072002001F021FE002805D4DA
:10A950000121002001F04AFE002800D50EE0002071
:10A9600002BD80B501464FF40072002001F023FEC5
:10A97000002803D401F001FE002002BD4FF0FF309B
:10A9800002BD10B5ADF5007D0446FCF7CBFC2028D8
:10A9900002D300F04BF803E000F072F8002802D573
:10A9A0004FF0FF3009E021466846FFF783FF21465C
:10A9B0004448FFF77FFF00F061F89DE080B5102864
:10A9C0003EBF13185B1E102B02D300F02FF8D5E703
:10A9D000BDE8084080009200203001F0D8BD70B57D
:10A9E00004461646102C3EBF3019401E1028ADF507
:10A9F000007D0D4602D300F019F803E000F040F8A6
:10AA0000002802D54FF0FF300DE0002007E0694636
:10AA1000021901EB820155F820200A62401CB04265
:10AA2000F5D300F02BF80DF5007D70BD072000F088
:10AA3000A9BCF8B504460D461F46032C3CBF781947
:10AA40004128ADF5007D164602D3FFF7EFFF03E086
:10AA500000F016F8002802D54FF0FF300BE00DEBA8
:10AA6000C4106D0800EB45003A4631466030FCF7F3
:10AA7000B7FC00F003F80DF5017DF0BD684670E706
:10AA800068465CE710B50446202221464FF4F0707A
:10AA900001F07DFD002800D516E02078FF2804BFD6
:10AAA0006178FF2908D1A078FF2804BFE178FF2949
:10AAB00002D103A001782170002010BD5858580021
:10AAC00000000000B14200204FF0FF3010BD10B573
:10AAD000ADF5007D0446FCF725FC202803D2FFF7E6
:10AAE000CFFF002802D54FF0FF3005E0214678A8BF
:10AAF000FFF7E0FEFFF7C2FF0DF5007D10BDA0F1EE
:10AB000030020A2A81B038BF30380CD3A0F141039B
:10AB1000062B38BF373806D3A0F16101062934BFB0
:10AB200057384FF0FF3001B07047F8B504460D4676
:10AB30000026207870B1617861B1FFF7E0FF074629
:10AB40006078FFF7DCFF00EB071005F8010BA41C91
:10AB5000761CEEE73046F2BD1FB50C4638494A6810
:10AB6000029220B1D1F8002037A100F02BFC6CB18B
:10AB70009DF808009DF80910019000919DF80A3099
:10AB80009DF80B2032A1204600F01CFC002004B0F0
:10AB900010BD000080B52B490A684B682FA100F05A
:10ABA00011FC002002BD1A2838BF413006D33428DA
:10ABB00038BF473002D33E2802D2001FC0B27047D0
:10ABC00001D140207047232070472DE9FC411D49E9
:10ABD0000A680092002749680191DDE900480B26C8
:10ABE0000546204641463E220023FCF74DFC104618
:10ABF000FFF7D9FFE855414620463E2200237F1C3F
:10AC0000FCF742FC761E04468846EAD102F01BF9A6
:10AC10000A2402F020F910F1010F03D1641EF8D1CB
:10AC2000FFF722FD3E22B0FBF2F23E2101FB1200B3
:10AC3000FFF7B9FFE855E91900204870BDE8F68133
:10AC400000010010600000106E52462578000000E0
:10AC500025632563256325630000000025303858EF
:10AC6000253038580000000030B5134B1C68202CEC
:10AC700008DA0C2565431D44641C1C6045F8040F6C
:10AC80006960AA6030BD2DE9FC410B4D0FF22C0824
:10AC900004462E1D002709E0B06800904146736805
:10ACA00056F80C2B2046FDF7B3F97F1C2868874225
:10ACB000F2DB0020BDE8F681106500206661756C4E
:10ACC00074203A2025642C2025642C2025640D0A4C
:10ACD0000000000000000000000000000000000074
:10ACE00010B5040008D000BF95A14FF47A4041F0A0
:10ACF00001018847641EF6D110BD00002DE9F04F18
:10AD000099B04FF0000818901791144616931698B2
:10AD1000804561D26078179915904144A0781490CD
:10AD2000E07813902079129060791190A279E379FC
:10AD3000267A677A94F80AC094F80BE094F80C50DD
:10AD400094F80D9094F80EA094F80FB05FA01091B5
:10AD500021780F911899F9B1CDF838B0CDF834A019
:10AD6000CDF830900B9505920693CDF828E0CDF8FC
:10AD700024C008970796119A12990F9B0492039189
:10AD8000139A1499029201910146159A009200209B
:10AD9000109AFEF79DFA1BE0CDF834B0CDF830A044
:10ADA000CDF82C900A95049205931199129A03916B
:10ADB0000292CDF824E01399149A01910092CDF8F3
:10ADC00020C0159B0F9A109907970696FDF7DDFF97
:10ADD000103408F110089AE7002019B0BDE8F08F90
:10ADE00070B504460129C0B088BF4FF0FF3019D8B4
:10ADF0000D0300264FF480726946284601F0C7FB18
:10AE000000280ED44FF480736A4631022046FFF7C3
:10AE100075FF0120FFF764FF761C102E05F5807585
:10AE2000E8DB002040B070BD2DE9F84F0D46032D42
:10AE3000C0B0834616460CD1706822A1FEF7BAFD59
:10AE400038B9B068FEF71CFD01465846FFF7C8FF49
:10AE500034E001270FF270080FF2CC092BE056F80E
:10AE60002700FEF70DFD8246BAF1000F25D45246A9
:10AE700049465846FDF7CCF8002404EB0A104FF47D
:10AE8000807269460002FFF732FA60B94FF48073AE
:10AE90006A4621025846FFF731FF0120FFF720FFE5
:10AEA000641C102CE9DB681E874203DA41465846D1
:10AEB000FDF7AEF87F1CAF42D1DB002041B0BDE80A
:10AEC000F08F00002D6900000D0A00002530345875
:10AED000203A202530325820253032582025303273
:10AEE000582025303258202530325820253032580D
:10AEF00020253032582025303258202D2025303260
:10AF000058202530325820253032582025303258EC
:10AF10002025303258202530325820253032582014
:10AF2000253032580D0A0000536563746F72202576
:10AF3000643A0D0A0A000000000000000000000052
:10AF40000338FDD87047000080B5002342F210722C
:10AF50000B49012001F08AFF0A4901220A7018B149
:10AF600000F010FA4FF0FF3002BD80B501F0C2FFD3
:10AF7000044A00211170F2E702480078704700008F
:10AF8000C9C80200566C0020F8B504460D46A2F16F
:10AF90000C07A0B0394605F10C0001F0D6FFA968F6
:10AFA0001FA6884207D000BF1FA3324600212046BB
:10AFB000FDF74CF825E06868042804D331462046A4
:10AFC000FDF750F81DE000973A46A868019005F19A
:10AFD0000C0102A8FCF714FA686807F108036A4636
:10AFE0000021FFF726FD002807D408A332460121DF
:10AFF0002046FDF72BF8002005E031462046FDF7FE
:10B0000035F84FF0FF3021B0F0BD0000534554003B
:10B010004B88012B08BFFFF7B7BF4FF0FF307047D9
:10B020004443464700000000435243204572726F7C
:10B030007200000070B4044604E015F8016BB342DE
:10B0400003D1641C23781BB10D462A78002AF4D161
:10B05000201A70BC704770B4044600E0641C23786A
:10B060003BB10D462A78002AF8D015F8016BB3429F
:10B07000F8D1201A70BC704718B40478954B1B5D4A
:10B080001BB118BC001D02F098B818BC0C3002F0BF
:10B090000CBB1CB50178904C002942D0022928D065
:10B0A00060D2017AD9B14168097804F1180002F040
:10B0B00041FC20B101218DF80010019006E0206ACA
:10B0C000616A081A05D000208DF800006846A16B5F
:10B0D0008847206AA18B626A101A814206D3012236
:10B0E00004F13D01201DFFF7C7FF13BD01202070B3
:10B0F00013BD8DF80010C068227976490190885CF4
:10B1000038B1012204F13D0104F1080002F055F8C4
:10B1100025E0012204F13D0104F1100002F0C5FA1E
:10B120001DE004F13C0104F1280002F016FC98B97E
:10B1300021796848405C38B1012204F13C0104F1F6
:10B14000080001F0E8FF13BD012204F13C0104F105
:10B15000100002F029FA13BD03208DF800006846A4
:10B16000A16B884713BD00002DE9F0475A4D0646F4
:10B170000C0088B01F46AA6308BF072050D0626841
:10B18000216892B205F1180002F0C0FB002847D1F7
:10B19000E268A16892B205F1280002F0B7FB00282E
:10B1A0003ED100BF4EA191E81C57684680E81C576D
:10B1B00071690691307C8DF81C70401E8041C0433F
:10B1C000C00F8DF81400707C00B10E208DF81500B2
:10B1D000424AF0680290B068039031680191694674
:10B1E00070680090281D02F0E4FBC8B92870306830
:10B1F00010F1010F13D02A793649885C38B1012249
:10B2000005F13D0105F1080001F0D7FF08E001223A
:10B2100005F13D0105F1100002F047FA00E00020C1
:10B2200008B0BDE8F08770B52B4C2678014604F1D4
:10B23000180002F092FB0546BEB10021217025489E
:10B240002179405C38B1012204F13D0104F108008C
:10B2500001F0B3FF06E0012204F13D0104F110000A
:10B2600002F023FA08B100F0CDF8284670BD70B5A1
:10B270000146194D05F1280002F05CFB040027D1BE
:10B280002979144E705C20B105F1080001F08CFFA3
:10B2900003E005F1100002F0CCF9C8B905F13C015A
:10B2A00005F1280002F059FB90B92979705C38B19A
:10B2B000012205F13C0105F1080001F02CFF06E038
:10B2C000012205F13C0105F1100002F06DF9044680
:10B2D000204670BDF06B0020A843002093B0020010
:10B2E000FFFFFFFFFFFFFFFFFFFFFFFFFFFFFFFF6E
:10B2F00000000000000000000000D6010601000070
:10B300001F480021016441648166C16600207047C6
:10B310001B494A6C01EB8203521C082A986428BF1F
:10B3200000224A640020704715490A6C486C82422A
:10B3300001D10020704701EB82004830521C082ADE
:10B3400028BF00220A6470470D48016C406C81429E
:10B3500000D1704780B5FFF7E7FFBDE8024002F07B
:10B360009DBB07498A6EC86E824201D1002070479A
:10B3700001EBC200521C082A28BF00228A667047CF
:10B380005469002001494865704700009842002038
:10B3900070B5054600262846FFF769FF78B10428F6
:10B3A0000DD1012406494FF47A4041F0010188474C
:10B3B000641EF7D1761CB6F5FA7FECDB0D2070BD6C
:10B3C000D00C03000CB430B583B0044606A802903C
:10B3D0000A4600250194009502AB01A9084878446B
:10B3E0001E30FAF70DFF01990D7000284EBF04467C
:10B3F0000198041B204603B030BC5DF80CFB00BF75
:10B40000D7BFFFFF18B583B0694600220023002490
:10B4100081E81C0002906A46002144F20100FFF717
:10B4200023FC04B010BD002818BF002901D10E2054
:10B4300070470278DE2A01D1082070470968416010
:10B44000DE2101704FF6FF7107E008B90E2070474A
:10B450000278DE2A01D00820704741800020704722
:10B460000246107A58B15088002166DF08B911727F
:10B47000704711281CBF516808470120107270479F
:10B48000F8B505460C0018BF002D84B04FD02078C9
:10B49000DE284CD1A9886088814204BF2046FFF78E
:10B4A000DFFF2888012805D0112839D051280FD076
:10B4B00005B0F0BD287A012802BFA98860888142C2
:10B4C00035D1012020722046FFF7CAFF05B0F0BD3C
:10B4D000A8886188884204BFA879022827D1A87B60
:10B4E00004281CBF0628052821D168460021002217
:10B4F0000023002680E84E004FF4C0700227ADF80C
:10B5000004008DF80070A87B052808BFADF8041072
:10B51000A8886946B0DF50B16168884705B0F0BDC2
:10B52000A8886188884204BF4FF6FF70608005B02C
:10B53000F0BDFEE730B505460C4687B0A1886869C6
:10B540006A4602F0D1FB182101A8FFF7AFF9029576
:10B55000A088ADF80C00009804902989E088884202
:10B5600004BF218A022913D1009808B304F1120004
:10B5700002F0E4FB20B1009901200870022102E0F2
:10B580000099087003218DF80410A96981B10DE0BC
:10B59000A98988420CD1A96951B100208DF8040015
:10B5A00004F112020592208AADF8180001A888471C
:10B5B00007B030BD38B505460C0018BF002D8AB065
:10B5C0005ED02888102805D0502836D057283AD089
:10B5D0000BB030BD002000906A46A988606902F077
:10B5E00083FB02A800210022C0E9001201A8022169
:10B5F000ADF808100390ADF80A202189A88802AAA6
:10B60000ADDF00283CD1A069002839D0039802F0B2
:10B6100095FBA8B3009808B101210170182104A876
:10B62000FFF744F902208DF810000594A888ADF8C2
:10B6300018000098079004A820E029462046FFF74C
:10B6400079FF0BB030BDA98860696A4602F04CFBF7
:10B65000B0B90098017800291CBFA06900280FD05C
:10B66000182101A8FFF722F901208DF804000294A7
:10B67000A888ADF80C000098049001A8A16988473B
:10B680000BB030BDF0B500BF4DA292E8E8008DB020
:10B69000040009A880E8E80014BF00290E2058D053
:10B6A0000868A061214609A862DF002851D12078EE
:10B6B0008DF802000121ADF80010A21C694601209E
:10B6C000A8DF002845D1202101A8FFF7EFF80220CC
:10B6D000ADF80400F4202178ADF808008DF80610CC
:10B6E00001219DF81100ADF80A1040F00C008DF812
:10B6F00011008DF810108DF815108DF8161004F14A
:10B700000C02608801A902F01FFB10BB202101A8D8
:10B71000FFF7CCF80320ADF80400F4202178ADF851
:10B7200008008DF8061001219DF81100ADF80A10EF
:10B7300040F010008DF811008DF810108DF81510E4
:10B740008DF816108DF81710221D608801A902F0DF
:10B75000FBFA0DB0F0BDF0B5040085B00D461646FD
:10B760001F4608BF0E2029D060696A46394602F09C
:10B77000BBFA18BB4FF6FF718F421ABF0098002822
:10B7800005201BD0007810B9082005B0F0BD318825
:10B79000F529A8BF072011DA01A800210022002303
:10B7A0008C4680E80E10A088ADF8040004950120B6
:10B7B0008DF80600039601A93846AEDF05B0F0BD4E
:10B7C0009ECADC240EE5A9E093F3A3B50000406E09
:10B7D000F8B486881746BC19B24228BF3746F51B15
:10B7E000C2881F4607EB020C934228BF1746D61BA0
:10B7F0004A8803889A4224BF4088904209D38888A7
:10B80000A84228BF844204D3C888B04228BF8445D8
:10B8100002D2F2BC00207047F2BC0120704738B55C
:10B82000804A04461089A1B288422BD17E4D107CFB
:10B83000297B88420FD202F11201A0B275DF30B12C
:10B8400011281CBFA96900291CD0884731BD107C74
:10B85000401C107431BD00211174287C48B13B217B
:10B86000A0B276DF002818BF082802D0A96901B16C
:10B870008847696931B100208DF80000ADF80240B9
:10B880006846884731BDF8B5010001D10E20F2BDF0
:10B8900091E8FC10644880E8FC10624C0460086881
:10B8A000A8B17ADFB8B9096820460822FBF798FDED
:10B8B0004FF6FF70208104F12000E06000215B4A18
:10B8C00004F10C0002F0AAFB28B10320F2BD2046CF
:10B8D0007BDF0028ECD0F2BD1CB50B460246597A3E
:10B8E000514C71B9187A002858680CBF6168A1687A
:10B8F00002F0A6FB00281CBFA16900290CD08847D4
:10B9000013BD00201872616931B101208DF800006B
:10B91000ADF802206846884713BD2DE9FC41044676
:10B920002088102807D011282FD0122861D0502845
:10B930003ED0BDE8F381E07BA58801286FD1394E68
:10B94000394F30894FF6FF78404519D100203074C7
:10B95000358106F1120031460822FBF741FD4346CE
:10B9600040F2F31204F1100106F11200FFF730FF6C
:10B970007074F889002852D106F1080128464BE07E
:10B98000B96900294BD0042030E0264DA1882889D0
:10B99000884244D1E86802F083FB00281FBF224997
:10B9A0008969002988474FF6FF702881BDE8F38137
:10B9B0001D4DE088E989884204BF208A022801BF22
:10B9C000A788184E3089B84229D104F1120002F03C
:10B9D000B5F918B106F1080138461DE0F06802F02B
:10B9E0005FFB00281CBFA969002918D0BDE8FC41F5
:10B9F00008470C4DA6882889B04210D14FF6FF7336
:10BA000040F2F31204F1080105F11200FFF7E0FE25
:10BA1000687405F108013046BDE8FC415CE7BDE80B
:10BA2000F3810000086A0020386B00201FB8020074
:10BA3000417949B100F22E41087828B98978481E29
:10BA40008041C043C00F70470020704780F830101D
:10BA50007047F8B504460D0018BF002C01D10E2028
:10BA6000F2BD05F17A000178012904BF807F012829
:10BA700031D005F19C07786804281CBF3968042977
:10BA800029D00020A07005F17801201D2C22FBF7A1
:10BA9000B7FC04F12406002030730721B868306138
:10BAA000F868706104F582674FF6FF70B8823F61F5
:10BAB00004F2264002F016FB207818B904F1500277
:10BAC000FF21117104F155003860307801280CBF56
:10BAD000EE201F2001E00720F2BDB88004F21442DE
:10BAE00004F15501284602F040FC28BB04F2312144
:10BAF000B96004F21C42307801280CBFEE201F20F0
:10BB0000B88105F13C0002F030FCA8B904F1500006
:10BB10000121417004F13C02A169B1840121317617
:10BB20000021F16101706069306204F1540072DF3C
:10BB300010B9012020700020F2BD00002DE9FC4169
:10BB400005460F46287810B90820BDE8F68105F2B1
:10BB50002648AF700721404602F0C4FAA87905F5DF
:10BB6000826605F1240410B1A978012906D0E8798C
:10BB700068B1A878012818BF022808D1216921B12D
:10BB8000012070770820884701E000207077F07D61
:10BB9000002804BF317E00290DD1707E002804BF2B
:10BBA000B17E002907D1F07E28B9317F481E80413F
:10BBB000C043C00F00E001207F1E032F18D8DFE82C
:10BBC00007F002090F13AA7922B1217811B938B10F
:10BBD00001200EE0E97900291CBF0028022008D1CD
:10BBE000287A08B1032004E0687A08B1042000E054
:10BBF0000020A870216981B1A878032818BF042803
:10BC00000BD16A794AB1B07F38B9002285F8302467
:10BC10000120F0770720884701E00020F077182105
:10BC200005F13C00FEF742FE0120207605F15007A9
:10BC3000A06801281CBF022801207870207828B154
:10BC4000616801291CBF02290121B97000213970E6
:10BC5000A978042943D8DFE801F074030F1F5100CD
:10BC600001206073002030612062C4F81C80022033
:10BC700020768020A08434E00221002814BF072011
:10BC80000320207661732869A08400203061C4F805
:10BC90001C80E868206224E0696921620028A969A3
:10BCA000A18414BF0620012020762846FFF7C0FE9D
:10BCB00090B1022038700122B188306802F091FC06
:10BCC00008B10421017005F13C02314605F1540030
:10BCD00072DF20B9052000E0032060733661A87888
:10BCE00088B3316905F13C0205F1540072DF78BB7D
:10BCF000217B387973DF30B3BDE8F681E9692162D1
:10BD00000028296AA18414BF062001202076284635
:10BD1000FFF78EFE98B1022038700122B18830689A
:10BD200002F05FFC08B10421017005F13C023146CC
:10BD300005F1540072DF0028D1D10620CDE70420A0
:10BD4000CBE700206073216909B1607B8847002040
:10BD5000BDE8F6811CB50C460188102904D01129D4
:10BD600009D0262914D013BDC17B01292BD180888D
:10BD7000A4F8240413BD04F2244100228A728088AE
:10BD80000988884204BF207900281CD101210FE0D6
:10BD9000007A012818BF022815D1A078401C81B272
:10BDA0004CF6CD424A43910C01EB8101401AC1B2DD
:10BDB0002046FFF7C3FE00281CBFA16B002902D05C
:10BDC000BDE81C40084713BD0249012081F8040169
:10BDD000704700BF80440020000000000000000009
:10BDE00080B5FDF78BFD1F491F4A0818506001BD43
:10BDF0007CB51E481C4D90F804012978814210D072
:10BE0000012828700DD100BF21A64FF4FA6446F036
:10BE100001064FF47A40B047641EFAD116A0FCF731
:10BE2000B4FF686840B1FDF769FD6968814203D2DB
:10BE300000206860FDF79EFA0D480E4A01681368FD
:10BE4000994205D0FFF770FABDE8764001F026BEB2
:10BE5000FFF792F8012803D1BDE8734002F0D2BB8E
:10BE600073BD000020BF0200086C00208044002049
:10BE70009469002098690020416E64726F69647E45
:10BE80007E7E7E7E0D0A0D0A00000000000000008C
:10BE90000338FDD8704700002028014604DA7348B3
:10BEA000C84000F001007047402808DA0122A1F1E3
:10BEB000200012FA00F018BF0120C0B27047012024
:10BEC000704700001FB5044678A1684602F0ADFB3C
:10BED00002E0684602F0BAFB029A3AB15168126871
:10BEE000204690470028F4D1112000E0002004B043
:10BEF00010BD00001FB504466FA1684602F095FB17
:10BF000006E05168126820469047684602F09EFBA2
:10BF1000029A002AF5D11FBD80B51620FFF7BCFF9D
:10BF200028B942F20100BDE80240FFF76BBA504861
:10BF300000784009082803D2EC21C140C80702D488
:10BF400042F20200EFE74B49886820B10A6842F4E8
:10BF500080020A6001BD48494FF48000086001BDBD
:10BF600080B51620FFF798FF28B9BDE8024042F2DD
:10BF70000100FFF747BA3F49886820B10A6822F4F8
:10BF800080020A6001BD3D494FF480000860BFF3A4
:10BF90004F8FBFF36F8F01BD3EB5394D287808B183
:10BFA00008203EBD0121A970FFF78CFF112820D089
:10BFB0000020FFF79FFF00BF45A00168019100220C
:10BFC0008DF80020684602F051FB2E4901A810DFD1
:10BFD0000446401E8041C00F00F034F80CB12046EA
:10BFE0003EBD0020A8706870FFF796FF0120FFF7A4
:10BFF00081FF00203EBD38B5214D287808B90820C2
:10C0000032BD0121A9700120FFF75CFF112817D074
:10C010000220FFF76FFF00208DF80000684602F055
:10C0200025FB11DF0446002000F00CF80CB120467F
:10C0300032BD0020A870FFF793FF0320FFF75AFFDF
:10C04000002032BD28709DF8000002F02BBB0C4888
:10C05000817809B9082070470078002818BFFFF7D9
:10C06000CABF99E70648007870470000FC06FFBD8C
:10C0700016E400E0CC6B002000E100E080E100E08D
:10C08000506C002069AC0200E0B500BF0DA168460D
:10C0900002F0CBFA05E0486809688847684602F074
:10C0A000D5FA02990029F6D107BDEDE7CC0A0300C5
:10C0B000DC0A030008000000DC0A0300EC0A0300AD
:10C0C00008000000EC0A0300FC0A0300080000005E
:10C0D000020000053EB50B00044601D10E203EBD16
:10C0E00041481860002168460022002580E82600AB
:10C0F000012028218DF800408DF80200ADF80410D1
:10C1000069461A68202069DF00F039F801208DF8AF
:10C110000100ADF8021069461A68402069DF00F09E
:10C120002EF8F7208DF80040ADF8020069461A6835
:10C13000232069DF684600210022002480E81600E1
:10C1400001208DF8000069461A6869DF00F011F8D7
:10C150004FF4B060009069461A68A12069DF00F0D2
:10C1600008F88DF8001069461A68A02069DF0020E1
:10C170003EBD68460021002280E8160070476846F0
:10C180000021002280E82600704760DF10B9174ABE
:10C190000121117070470000144900B50878ADF511
:10C1A000017D88B903E0052818BFFFF72BF90DF5CD
:10C1B000017D00BD5168126804A8904701A802F0F3
:10C1C00045FA039A002AF5D14FF4FA70ADF8000051
:10C1D000694604A861DF0028E5D100BF04A101A8D9
:10C1E00002F023FAEDE7000000400020536C00202D
:10C1F000A80B0300C80B030008000000F721018012
:10C2000017214180002101714171FB2181711B21A6
:10C21000C171704730B400BF6EA284B0D2E900454E
:10C22000CDE90045ADF80010ADF8021067A1D1E9E5
:10C230000023CDE90223694602AA21E008B90E20B5
:10C2400070470161F72101804180FB210171F721D5
:10C25000C1801721018100218172C172FB2101730C
:10C260001B2141730020704708B90E207047A1F1CF
:10C270001702E12A01D30720704701800020704790
:10C2800090DF04B030BC7047F0B502468BB09088A8
:10C2900000280C4640F09880118810290BD01129F5
:10C2A00019D0232900F07D8024295DD03A2916D0A9
:10C2B00055293AD07FE0A01D21798171D27B012AD6
:10C2C00003D0022A03D1628800E022880280C0796C
:10C2D000884270D26CE0A01DFFF790FF6BE0A51DB7
:10C2E00050892988884228BF0846688068881728AE
:10C2F000B8BF17206880216900291CBF6879002811
:10C300000FD000BF35A10020D1E90023CDE90023E3
:10C31000ADF8020069466888ADF80400204622693D
:10C32000904700206871287145E0D088A21D172829
:10C330001188B8BF1720884228BF084650800020C7
:10C340001071B5DF5179002935D12069002832D02C
:10C3500024A10020D1E90067CDE90067ADF8020013
:10C360005088ADF8040017E0111D68462C22FBF739
:10C3700047F8BDF80010BDF8040004EBC10250738B
:10C380002069C0B119A3D3E90067CDE90067ADF812
:10C390000210507B8DF804006946226920469047C0
:10C3A00009E0A01D12898179D2B2914288BF11465D
:10C3B0000020FFF72FFFA07A30B1E1880020A5DF31
:10C3C00010B9A0720120E0720BB0F0BD00000000B7
:10C3D000000000000000000000000000770A0000DC
:10C3E00000000000770A0000000000007ADA000078
:10C3F0000000000012F003030FD1094B9A6001F115
:10C40000010C4FEACC4C02EB1C42DA6000225A705D
:10C410001A705880998000207047072070470000EC
:10C42000BC6B002080B5FAF77DFF801C032190FBD8
:10C43000F1F0800002BD00002DE9FC420500144629
:10C4400018BF002C89461E4603D0FFF7EBFF86423B
:10C4500041DA00203DE0021D954249DB9CF80020B6
:10C460009208B25C0A5438469CF800709CF801208F
:10C470003F0107F0300747EA22171A19F75D0F54FA
:10C480001F197F789278BF0007F03C0747EAA21790
:10C49000401CF75D0F54401C1F19E41CBF7807F0C7
:10C4A0003F07F65D0E54401C1AE01A192D01527810
:10C4B00005F0300545EA22151A19755DCD555278FB
:10C4C00002F00F0216F822300B54401C3D220A5491
:10C4D000401CBDE8F6822B4621463546002400204C
:10C4E000471CA9F10202944203EB040C0BA6B2DB39
:10C4F0004C45EEDA9CF80050AD08725D0A54781C89
:10C50000A9F101029CF800509442CED105F0030538
:10C510002D01725DCA553D220A54D6E75137535456
:10C5200066696A6768775A306E5770715573494A01
:10C53000364C4142797A44434533474875345978FB
:10C540004D39504F6164386272566F586B6C6D3163
:10C55000324676354B52634E74652B2F0000000037
:10C56000704780B500222D492D4802F0B5F818B16A
:10C57000FEF708FF4FF0FF3002BD10B5284C00E079
:10C5800041DF204602F02AF90028F9D110BD80B51C
:10C590001346B0F5005F3EBF1A18521EB2F5005F99
:10C5A00006D200F01EF802F0A2F818B1FEF7EAFE7B
:10C5B0004FF0FF3002BD80B51346B0F5005F3EBFBF
:10C5C0001A18521EB2F5005F08D20022009200F045
:10C5D00008F802F0AFF818B1FEF7D4FE4FF0FF30C4
:10C5E00002BD0A4600F5D0210D48704780B50A46C5
:10C5F000B0F5005F3EBF00EB0231491EB1F5005FB0
:10C6000008D200F5D0210023054802F0C3F818B184
:10C61000FEF7B8FE4FF0FF3002BD0000C80B03006C
:10C620006C4400200C48006870470B48016840F6D5
:10C630004C12914201D36420704740F2C67081428F
:10C6400001D200207047A1F2C671642041434FF42B
:10C65000C372B1FBF2F07047D840002010B5044619
:10C66000FAF7ECFD01462046096ABDE8104008478C
:10C6700010B50446FAF7E2FD01462046896ABDE896
:10C68000104008470000000000000000000000000B
:10C6900028B10FF2EC01800141F001010847704719
:10C6A000C1888289491CC18089B2914210D1002180
:10C6B000C1808188C289491C818089B2914207D199
:10C6C00000218180428841898A4208BF491C4180FB
:10C6D0007047F8B505460C462889012816461F46BE
:10C6E00005D1FDF757FE012811D002202881A98825
:10C6F000002904BFE88800280FD1288948B9688834
:10C700003946FDF754FE012F07D101202881112061
:10C71000F2BD022804BF00202881FDF7EFF807468C
:10C7200068882B88000300EB0340AB88214600EBB0
:10C7300003202C8AEB88B2B203FB0400FDF796FEBF
:10C7400004464620FFF7A4FFFDF7D8F83946FDF769
:10C75000D8F8C928084E02D33088401C30802846BB
:10C76000FFF79EFF0CB90020F2BD3088401C3080DE
:10C770002046F2BD000000006A6B002000000000AF
:10C780000338FDD8704700000000000000000000E2
:10C7900028B10FF22C11800141F0010108477047C8
:10C7A000C1884289491CC18089B291421BD30021B2
:10C7B000C1808188491C818089B2102913DB002146
:10C7C00081804188491C418089B210290BDB0021FE
:10C7D00041800188491C018089B2C289521C914262
:10C7E000A4BF81890180002070474620D0E7F8B5BA
:10C7F00005460E4628890128144605D1FDF7CAFDD5
:10C8000001281CD002202881A988002904BFE888BB
:10C8100000281CD12889B0B9EB8969882A889A42F6
:10C8200008BF0F2901EB021002D10121102002E004
:10C83000401C012180B2FDF7BAFD012028811120A2
:10C84000FEF7A0FD2DE0022804BF00202881FDF79F
:10C8500055F807466B88288831461B03AE8803EBE2
:10C860000043E888A2B203EB062300FB0434204611
:10C87000FDF7FCFD0446FDF741F83946FDF741F8A8
:10C88000C9280A4E02D33088401C3080FFF7ADFF24
:10C890002846FFF785FF0CB90020F2BD3088401C08
:10C8A00030804FF0FF30F2BD000000006A6B0020C6
:10C8B0000000000000000000000000000000000078
:10C8C0000338FDD87047000070B53B4C3B4D2068E5
:10C8D000401CC107206032D5686801F0B6FF0646EB
:10C8E000E06B308040F6FF7188420CBF0120401C95
:10C8F000E063206C18B1328831490A433280207DD0
:10C9000018B1318841F4804104E0607D18B131886C
:10C9100041F400513180B01C01F0BDFF38B9B01CAA
:10C920000020C04638B1C0B202F012F803E03088EF
:10C9300040F480503080686801F089FF06E0296883
:10C94000884203D30A31296002F046F81D48016885
:10C9500000291DD5FDF71EFD012819D0206861684A
:10C96000884208D30120FDF764F888B9606800F6B2
:10C97000B830606070BD686801F072FFA86038B1BF
:10C98000FDF788F920B96868BDE8704001F072BF12
:10C9900070BD09490A686423B2FBF3F3642000FB0D
:10C9A00013234D2B02D24D32D21A02E06432D21A36
:10C9B0004D324A607047000098420020F842002043
:10C9C0000080FFFFD0400020CB074CBF092300238D
:10C9D000D380C1F34303C1F343119380518010808E
:10C9E00070472DE9F04104463C4F208878809846F6
:10C9F000B980154660882388000300EB0340A388B4
:10CA0000E4880E2600EB03207E22B91D06FB0400FD
:10CA1000FDF76DFC002807D4B7F90610002904BF04
:10CA2000B7F90800002802D14FF0FF300EE0012DC9
:10CA300004D100F035F84643B61D00E08426424696
:10CA4000B1B23846BDE8F041FCF7F5BBBDE8F08176
:10CA50007CB515460C461E466A46FFF7B5FF3346C1
:10CA60002A4644F400416846FFF7BBFF76BD38B55F
:10CA700004461B481B4A13680D46016899420DD0B5
:10CA8000FEF76FFC0168042906D14068010C2B46B3
:10CA9000224680B2FFF7DCFF012032BD002032BD0C
:10CAA00010B500203E210D4A02EB4103B3F90640C8
:10CAB00014F1010F02D1401C491EF5D50721B0FB2E
:10CAC000F1F0C0F1090010BD024604484FF6FF71B5
:10CAD000418081800621FCF7AEBB00001C41002094
:10CAE000BC690020C06900200000000000000000B8
:10CAF00030B5039D049C41EA420141EA830141EAC9
:10CB00000521354A41EA044142F8201030BDE0B524
:10CB100000210191009100230122012105E0E0B5EF
:10CB20000B460021002201910092FFF7E1FF07BDB3
:10CB300080B51920FFF7EBFF1A20FFF7E8FF1F2051
:10CB4000FFF7E5FF1E20FFF7E2FF1D20FFF7DFFFE5
:10CB500000210220FFF7E3FF00211B20FFF7DFFF8A
:10CB600000211C20FFF7DBFF002002BD1B4900E075
:10CB70001B494FF0007008607047184900E01849E1
:10CB80004FF080600860704714494FF00040086023
:10CB90007047124900E012494FF08040086070472A
:10CBA0000E49FFE74FF00050086070470C484FF007
:10CBB000804101604FF0005101604FF00041016081
:10CBC000704708480068C00E02E006480068000F81
:10CBD00000F00100704700000007005008050050F9
:10CBE0000C0500501005005000000000000000007F
:10CBF00038B400F5A36210688DF800008B69486AAC
:10CC0000984203D29DF800304C6923544B6A91F846
:10CC100028005B1C4B625C1C48B10869844298BFC9
:10CC2000204608618869844298BF20468861086967
:10CC3000844203D2C868005D50600DE08D69AC424B
:10CC400003D291F82000506006E0834204D3AB4247
:10CC500032BC8041C00F704732BC01207047F8B52C
:10CC60000579434C2C2313FB05F52C440025667FE6
:10CC70000EB11120F2BD23680BB10126667704F1D5
:10CC80000C0391E8C05083E8C050A37F84F828507B
:10CC9000FF2B04D0012606FA03F3364E736012B15F
:10CCA0006577062540E00668656206F54172042056
:10CCB0005060C6F80851D6F808010090009B4868FB
:10CCC00000281ABF0B68187894F82000C6F81C05D5
:10CCD0004868022804D309684878C6F81C0506E0AD
:10CCE000C868022824BF94F82010C6F81C152068D4
:10CCF00010B10421116017E0D6F808010028FBD01C
:10CD0000C6F80851D6F8080100903046009921462F
:10CD1000FFF76EFF0028EFD1A07FFF2804D001218C
:10CD200001FA00F0134908602846F2BD1CB512480C
:10CD30000F4C002101600068009000990F482146C7
:10CD4000FFF756FF90B9A07FFF2804D0012101FA18
:10CD500000F008490860002060772072616822684E
:10CD600004F1080002B0BDE81040104713BD0000F8
:10CD7000786A002008050050083102400030024067
:10CD80001CB5049C0094001D02F043F816BD38B594
:10CD90000446012000900D462046FFF7F1FF30B910
:10CDA000059B049A2946201D02F04CF818B1FEF7A5
:10CDB000E9FA4FF0FF3032BDF0B585B00024002510
:10CDC00001AE05E0102C18DA575D3755641C6D1C58
:10CDD0009D42F7DB0B9A0A9B002595420FDA102C37
:10CDE000BFBF5F5D3755641C6D1CF6DB05E0FEF7C9
:10CDF000C9FA4FF0FF3005B0F0BD0720F7E7012278
:10CE00000092E3B201AAFFF7BBFF0028EFD1F2E7DF
:10CE10000000FEE700B500BF1300964694461039A7
:10CE200028BFA0E80C50FAD85FEA417C28BF0CC0AC
:10CE300048BF40F8042BC90728BF20F8022B48BF81
:10CE400000F8012B00BD80B5002002F09FF808B16A
:10CE50004FF0FF3002BD80B50421684602F0BAF8F9
:10CE600008B9009802BD4FF0FF3002BD2DE9FC4724
:10CE700004460F46380091461E4608BF0E2037D0A4
:10CE8000012C07D14FF00108214D687850B90820D6
:10CE9000BDE8F687200008BF4FF48078F4D0072063
:10CEA000BDE8F68703280FF26C0A05D1504602F060
:10CEB000FAF80220687001E0022802D1504602F020
:10CEC000F6F82C706F60AE600120009043464A4631
:10CED0000021504602F009F968780228504602D134
:10CEE00002F0DDF801E002F0CDF8032068700020C8
:10CEF000BDE8F68710B5064C6178032905D100BF5F
:10CF000004A002F0D0F802216170002010BD0000E2
:10CF1000E46B0020009000400104000018B50021DF
:10CF2000174A0B4608205C08DB07234644BF154C14
:10CF30006340401EF7D142F82130491CB1F5807F93
:10CF4000EFD311490120086011BD70B50D460E499F
:10CF5000044608684FF0FF3608B9FFF7DFFF0020EE
:10CF6000074908E0225C724002F0FF0251F82230CB
:10CF700083EA1626401CA842F4D3F04370BD00009B
:10CF8000106100202083B8ED2C6C002018B40A68D2
:10CF900012F1010F0BD0012303FA02F2DFF854342F
:10CFA0001A60DFF854340C68032243F824204A68DE
:10CFB00012F1010F04D0DFF84044002344F822307E
:10CFC0000268886902F2245318604C7D087D04438E
:10CFD0009C6448680B6802F20C542360A060087DD2
:10CFE00001281ED1886810F1010F04D0DFF8084431
:10CFF000002344F82030C86810F1010F0BD0012342
:10D0000003FA00F0DFF8EC331860DFF8EC33CC689B
:10D01000032043F8240002F5A1628868C968116002
:10D02000906011BC70470000F8B504460E462179A7
:10D03000DFF8C803174601EBC10200EB820595F843
:10D04000200008B10820F2BD0FF2C832206852F863
:10D05000211002F0A0F808B11120F2BD314620469F
:10D06000FFF794FF6F60306928606868002845D03A
:10D070002068317F0022C0F810214901D0F810212A
:10D0800000920022009BC0F82021D0F820210092BD
:10D090000022009BC0F82421D0F824210092002215
:10D0A000009BC0F84421D0F8442100920022009B4C
:10D0B000C0F85821D0F858210092009BDFF8402397
:10D0C000C0F8042300030016002803D4DFF834233B
:10D0D000115406E0DFF8302300F00F00104400F890
:10D0E000041C21680903091608D4012201F01F005D
:10D0F000DFF818338240490943F8212021680820CD
:10D10000C1F800050020A861E8616861012085F888
:10D1100020000020F2BD78B40479DFF8E03204EB9F
:10D12000C40503EB850301F06045B5F1005F1C46C3
:10D130002AD15B695BBB6261A1600021056805F5CE
:10D140009073196018680090009AC5F85811D5F8C6
:10D1500058010090009A6069A66805F24452166072
:10D1600050600120A8606068D8B91A68501E8041DC
:10D170009A6BC043521E9241D243D20F52EAD070F2
:10D18000F3D03AB10F210AE072BC1020704772BC94
:10D19000112070470120E860986B0028FCD0002225
:10D1A0006261084672BC70470079944900EBC00286
:10D1B00001EB82014B69581E81E02DE9F8410346DD
:10D1C0008E4E187900EBC00406EB840C0F4607F076
:10D1D0006044B4F1005F1AD1DCF80400002538B1D6
:10D1E000D3F800E00EF541784FF40474C8F8044019
:10D1F000DCF818409CB1DCF81C505DB120B1196816
:10D200004FF40470C1F804031120BDE8F28110202E
:10D21000BDE8F2810125CCF81010104604E0CCF8EE
:10D220001820CCF80C100020CCF81C000024196841
:10D2300001F5887ECEF80040DEF8000000900098EE
:10D24000C1F84441D1F844010090009801F23450F3
:10D250000760426015B90120086005E0D1F80002BE
:10D2600040F02000C1F800021A7902EBC2008300EE
:10D27000301DC058E0B9DEF80010481E8041DEF8CD
:10D280003410C0434A1E9241D243DEF81410D20F2C
:10D29000491E8941C943C90F42EAD0700843EAD008
:10D2A00006F11805EC5001B103242AB10F2403E064
:10D2B0004FF40470C1F804032046BDE8F2818041B8
:10D2C000C043C00F704780B584B00346012002916F
:10D2D0008DF800000192684619685A680DE080B523
:10D2E00084B0024600208DF8000002910021906871
:10D2F00001905161684611685268904705B000BDC1
:10D3000078B5044604F5887685B00D467169D9B9BB
:10D310003068002836D03160316800910098D4F828
:10D320003C15A86981422DD1EA68E86930B3D4F888
:10D33000003223F02003C4F80032E869A8612869AC
:10D34000E8600020E8611AE00020706170690090D8
:10D35000022000998DF804000021D4F88004C4F85C
:10D3600080040490D4F83C050390E8680290A96119
:10D37000E96101A829686A68904703E0A861284626
:10D38000FFF7A1FF706B78B100217163706B0090A3
:10D390000099A86940B10021A961E9612846D4F843
:10D3A0003C15EA68FFF78FFF306970B100213161E9
:10D3B0003069009001200099E060686928B104F2AA
:10D3C0003C5128460969FFF78AFFB06C60B1002123
:10D3D000B164B06C00900099686928B104F23C51C6
:10D3E00028460969FFF77BFF06B070BD034908486E
:10D3F00086E700000805005000070050F46A00208E
:10D400001003420000E400E018ED00E000E100E05D
:10D4100000200040EDD3020018B40A6812F1010F99
:10D420000BD0012303FA02F2DFF8BC341A60DFF8F4
:10D43000BC340C68032243F824204A6812F1010F1F
:10D4400004D0DFF8A844002344F822300268886939
:10D4500002F2245318604C7D087D04439C644868A4
:10D460000B6802F20C54A0602360087D01281ED1D5
:10D47000886810F1010F04D0DFF87044002344F8ED
:10D480002030C86810F1010F0BD0012303FA00F01F
:10D49000DFF854341860DFF85434CC68032043F8C4
:10D4A000240002F5A1628868C9681160906011BC0F
:10D4B000704700002DE9FC4104460F469046217953
:10D4C000DFF82C042C2212FB01F2851805F1290645
:10D4D000707810B10820BDE8F6810FF22C42206868
:10D4E00052F8211001F057FE00B19FE03946204666
:10D4F000FFF792FFC5F8048038692860686880B338
:10D500002068397F0022C0F81C214901D0F81C2175
:10D5100000920022009BC0F84421D0F844210092E0
:10D52000009BDFF8D023C0F8042300030016002876
:10D5300003D4DFF8C423115406E0DFF8C02300F061
:10D540000F00104400F8041C21680903091608D4D0
:10D55000012201F01F00DFF8A8338240490943F897
:10D56000212021680420C1F800050020A861E8619D
:10D5700030706861012070700020BDE8F68181B0D4
:10D580000022C0F81C21D0F81C210092009B8A6860
:10D590000B6AD25CD1F820C00CF1010CC1F820C09C
:10D5A000C0F81C2501B070472DE9FC4104462C2031
:10D5B0002579DFF83C3310FB05F51D446869B8B9DF
:10D5C0006A61A960286285F8280000262068C0F8F2
:10D5D0001C61D0F81C1100910121009A816029463C
:10D5E000FFF7CDFF686860B9D4F800806F690FE07D
:10D5F0001CE0D1F81C010028FBD00122CA600020E9
:10D6000068613046BDE8F68129464046FFF7B7FF1E
:10D61000286A2168B842ECD2D8F81C110029F3D14D
:10D6200095F828000028F7D00F26E8E71120BDE87C
:10D63000F6810279DFF8B8122C2010FB02F288186C
:10D640004169A2E081B000680021C0F82411D0F83F
:10D65000241100910021009AC0F80811D0F8081197
:10D6600000910121009A016001B0704781B08A6980
:10D6700052B90021C0F80811D0F808110091009AA1
:10D68000D0F8180501B070470022C0F80821D0F882
:10D6900008210092009B4A6AD0F81805CB6898547C
:10D6A000486A401C486201B07047F8B506462C2015
:10D6B00034798F4B10FB04F41F190023786828B1CC
:10D6C000356805F541704FF401744460B86970B174
:10D6D000FB6943B1786820B132684FF40171C2F838
:10D6E00004131120F2BD01233961FA6103E0BA612C
:10D6F000F9607862F86197F82900034304BF304667
:10D70000FFF7A0FF78683168002838D10022C1F8FF
:10D710004421D1F8440100900099326802F58471E7
:10D72000C869441EA441E4430868C96BE40F401E65
:10D730008041C0434D1EAD41ED43ED0F45EAD07031
:10D740002043EAD055EA040007D139461046FFF7D6
:10D750008DFF786AB9698842DFD30020B8610CB1C7
:10D760000320F2BD0DB10F20F2BD97F829003168FA
:10D77000002807BF01224A6001220A6003E04FF43B
:10D780000170C1F804030020F2BD481E8041C0436F
:10D79000C00F704780B584B00346012002918DF818
:10D7A00000000192684619685A680DE080B584B09F
:10D7B000024600208DF8000002910021906801903F
:10D7C0005161684611685268904705B000BDF0B5D8
:10D7D00085B00D46044604F5417704F58476386833
:10D7E000810523D5F06908B30021F16105F1280214
:10D7F000F06900904FF4017000997860507808B992
:10D800000121616002208DF804000021D4F8800419
:10D81000C4F880040490A8690390E8680290A961A4
:10D82000E96101A829686A68904727E039684807D4
:10D8300024D5306810B329462046FFF717FFA869A2
:10D84000696A88421AD1E86940B1EA68696AA861E0
:10D850002869E8600020E86168620CE005F12801B1
:10D86000487808B9012161604FF4017078600020A8
:10D87000EA68A861696A2846FFF78CFF7069B0B151
:10D880006869296A814207D295F8280020B929469B
:10D890002046FFF774FE0AE0002171617069009074
:10D8A0000099686918B169692846FFF77FFFF06B36
:10D8B00098B10021F163F06B0090009905F1280107
:10D8C000487808B101212160A86930B10021A9611F
:10D8D0002846EA68696AFFF75DFF05B0F0BD0449B4
:10D8E000084874E7000000000805005000070050D9
:10D8F000A46A00208000020000E400E018ED00E0CF
:10D9000000E100E000200040DFD8020009B90E204D
:10D910007047130004D0A2F1010C1CEA020F01D0E1
:10D92000092070470160511E818000218160C16023
:10D930000020704783688288D0F80CC0ACEB0303EA
:10D940009A4208D30368D0F80CC002EA0C0299543A
:10D95000C168491CEBE7042070478268C3689A1AC3
:10D960000BD00368D0F808C0828802EA0C0C13F8C8
:10D970000C300B708168491C01E005207047816004
:10D980000020704780B500E080B584B002788DF843
:10D9900000204368019382688DF80820C068174A08
:10D9A000039002EB8102684691685268904705B087
:10D9B00000BD2DE9F84F88B00378104C04EB8305C7
:10D9C0006A600E69AE604D7FE5546D4691E8C05FB8
:10D9D00085E8C05F04930378E15C31B102B1084A85
:10D9E0006946001DFFF720FB05E002B1054A6946C4
:10D9F0000C30FFF75FFD09B0BDE8F08FF06B002041
:10DA000085D9020089D90200000000000000000052
:10DA100028B100BFB2A1800141F001010847704761
:10DA200010B5040005D04FF47A70FFF7F1FF641EC3
:10DA3000F9D110BD2DE9F0410E4600270FF2FC1878
:10DA400037704146FBF700F905467DA1FBF7B2FFB1
:10DA5000441EA441E40FE5B1002F02DD414600F071
:10DA60001AF8032F0BD0042F07D134B1794801687D
:10DA700000F011F873A100F00EF8294600E0764995
:10DA800000F009F841460020FBF7DEF87F1C054650
:10DA9000E1E7BDE8F081304601F09EBB30B5ADF561
:10DAA000117D00686D4C401E072867A551D8DFE83E
:10DAB00000F00451C1C1A0A7AABAFBF75FF9014663
:10DAC00051A8FCF7F7FEFBF75BF951A801F094FBB6
:10DAD0005FF0040266A100F0C7F850BB2C2151A8EA
:10DAE00001F09FFB040006D0214603A8FCF7E2FEEC
:10DAF0000020207004E0032254A103A8F9F780FC61
:10DB00000CA8FDF747F807A8FBF704FC03A807A932
:10DB10000CAA534B02900191009251AAD3F8003005
:10DB200055A111A8FDF74EFC51A911A8FFF782FFDE
:10DB30000AE0022246A100F097F828B911A951A8DD
:10DB4000FFF778FF11AA00E051AA29460020FBF751
:10DB5000BFFB6FE0FBF764FB014651A8FCF7AAFE90
:10DB6000FBF764FB5FF0070249A100F07DF8002895
:10DB700060D0052248A100F077F828B9FBF752FBE6
:10DB800052A9421F491C20E05FF0070244A100F0A7
:10DB90006BF8B0B15FF0070243A100F065F880B107
:10DBA0005FF0090242A100F05FF850B15FF0090296
:10DBB00042A100F059F820B143A151A8FBF7FAFEA9
:10DBC00038B9FBF72FFB024651A90120FAF74EFEA8
:10DBD00030E051A8F9F7A6FB51A9084410F8010C50
:10DBE0000D2816BF0A2828460FF2E400FBF7CDF8EF
:10DBF00020E041F29410FFF70BFFFEF7CAFF19E097
:10DC0000FBF71EF916E043F69820FFF709FF002006
:10DC1000A075144890F8041101290CBF01200420BC
:10DC200001F060FC06E04FF47A70FFF7F9FE206C1B
:10DC3000FBF72EFC00200DF5117D30BD3B000000F0
:10DC4000513D31003A000000257300002D310000E5
:10DC5000513D0000D4400020B142002098420020F5
:10DC60003C6C00208044002051A801F0C5BC00009D
:10DC7000513D313B0000000025732C253038582CD5
:10DC800025732C257325732C312C303B300000007C
:10DC9000416E64726F6964004E52463E200000007F
:10DCA000736574206964200073686F77206964006D
:10DCB000736574206E616D652000000073686F7776
:10DCC000206E616D65000000636C6F73650000007D
:10DCD00025730D0A00000000000000000000000095
:10DCE0000338FDD87047000038B5054614001EBF44
:10DCF00000202060002D01D0286808B90E2032BD18
:10DD0000E888420800EB92729208B0EB820001D0E2
:10DD1000072032BD084601F02BFDC0B2142801D106
:10DD2000052032BD2979884201DB042032BDE98813
:10DD30002A68484310442060002032BD0078FFE785
:10DD400000F0010070470000F8B50F4690B005469E
:10DD5000B878164600B901208DF80E0003213888E6
:10DD6000ADF80C0001A8FCF7A1FD787C401E002155
:10DD700004288DF8041011D8DFE800F00D0907051C
:10DD80000300222008E0122102E0312004E02121DA
:10DD90008DF8041002E011208DF80400B87C401EBC
:10DDA000002104288DF8051011D8DFE800F00D09D6
:10DDB00007050300222008E0122102E0312004E0E0
:10DDC00021218DF8051002E011208DF80500F87B67
:10DDD0009DF80610421E9241D24301F0F701D20F86
:10DDE00041EAC2018DF8061001F0EF01387C421EB5
:10DDF0009241D243D20F41EA02118DF8061001F090
:10DE0000FE013A7B501E8041C04341EAD0718DF83B
:10DE1000061001F0F901387D002814BF022001200E
:10DE200041EA40018DF8061009A81C21FCF73EFDCF
:10DE3000787B10F0300F29D0032102A8FCF736FDC3
:10DE4000F87C401E002104288DF8091011D8DFE865
:10DE500000F00D0907050300222008E0122102E06E
:10DE6000312004E021218DF8091002E011208DF805
:10DE700009009DF80A0000F0F90040F002008DF85A
:10DE80000A00112102A88DF808100E90787B8DF8F9
:10DE9000240004A8B97B8DF825101421FCF706FD99
:10DEA00003A8049001A90591B888ADF81C00B868D2
:10DEB00018B1F988ADF818100890BC69002C71D021
:10DEC00003216846FCF7F2FC2088ADF82C00002105
:10DED0006088ADF82E0060680A90CDF834D0207BC1
:10DEE0008DF80010401E042811D8DFE800F00D095D
:10DEF00007050300222008E0122102E0312004E09F
:10DF000021218DF8001002E011208DF80000B96980
:10DF1000487B401E002204288DF8012011D8DFE83C
:10DF200000F00D0907050300222008E0122102E09D
:10DF3000312004E021218DF8011002E011208DF83C
:10DF40000100B869817A481E80419DF80210C043E3
:10DF5000C00F01F0F70141EAC0018DF8021001F095
:10DF6000EF01B869C27A501E8041C043C00F41EA38
:10DF700000118DF8021001F0FE01B869027A501EFE
:10DF80008041C04341EAD0718DF8021001F0F901DF
:10DF9000BA69907B002814BF0220012041EA4001A9
:10DFA0008DF80210F86900B10C90334604AA09A953
:10DFB0002846AADF11B0F0BD10B5DFF8244104F106
:10DFC0001C0001F0EDFBD4E9022300211018594197
:10DFD000D4E90423994206D828BF904203D2B0F175
:10DFE0007F4061F1FF3110BD7CB504460D463C4ECB
:10DFF000694606F17C0001F02BFC68B104704560B5
:10E00000694606F17C0001F04BFC18B106F11C00DA
:10E0100001F0CAFB002076BD042076BD10B41300C9
:10E0200008BF07200AD000684FF0FF34C0E902445F
:10E03000012918BF002142610161002010BC704716
:10E040002DE9FC410E46002105468DF80010904652
:10E05000684600F00BFBD5E902234FF0FF30834206
:10E0600008BF824208D1FFF7A7FF00278019794136
:10E07000C5E90201012400E000249DF8000000F041
:10E0800011FB14B90020BDE8F6812869C5F8188095
:10E0900000B12E6129460020FFF7A6FFBDE8F681FA
:10E0A00038B5002105468DF80010684600F0DEFA0C
:10E0B000D5E902234FF0FF30834207BF824200249C
:10E0C000C5E9020001249DF8000000F0EBFA0CB94C
:10E0D000002032BD29460120FFF786FF32BD000037
:10E0E00000400020002201F025BC78B405460C4613
:10E0F0002978012902BF68780028072045D01088B8
:10E10000861CB3422ED3012904D169784118891C99
:10E110008B4227D31B1A9B1E9BB2ADF80030694679
:10E1200010882044801C7DDF78BB2878022804D02A
:10E130006978BDF80060B14205D3BDF800108B428C
:10E14000A8BF09210ADA0821012805D1687883428D
:10E15000A8BFADF8000001DAADF80030BDF800004E
:10E16000FF2802D372BC0C2070471388401CE05477
:10E170001088401C108080B221541188491C1180E5
:10E18000BDF8000041181180002072BC70472DE9D5
:10E19000FC470A9FDDF82C803D881C46002306467C
:10E1A0008A46964699461DE039889DF80020521807
:10E1B0001018804538DB43B9491C3980012389B2E6
:10E1C00004F801A03888401C388069463A88224407
:10E1D00001A864DFE8B939889DF800000818388084
:10E1E00009F101093088814515DA706850F8290075
:10E1F00001900022694601A864DF50B99DF8000033
:10E200007045EDD1002B14BF00200220CCE76055F3
:10E210000020BDE8F687002BFAD03888401B401E4E
:10E2200081B2B1F5807FF2DB0C20BDE8F6872DE9E5
:10E23000FC41089F099C01941646054698460097A4
:10E240000222FFF7A4FF38B9019400974346102239
:10E2500031462846FFF79BFFBDE8F681F0B41488ED
:10E26000A51DAB4238BF0C2014D30388062B10DB4E
:10E2700040F68146B34203DB4FF6FF77BB4208D13D
:10E280004588062D05DBB5424FF6FF7704DBBD421E
:10E2900006D00720F0BC7047BB4201D09D42F8D3A6
:10E2A00005230B55122413885B1C13809BB2CC549E
:10E2B00013885B1C13809BB20B4404881C70240AD7
:10E2C0005C7013889B1C13809BB2194440880870B3
:10E2D000000A48701088801C10800020F0BC704735
:10E2E0002DE9FC4100F12807884638681646B0B38E
:10E2F000002523E03188401C08F8010016213088F1
:10E30000401C308080B208F800103088401C3080FB
:10E3100080B2404421880170090A41703088801C15
:10E320003080A2884AB1A168C9B180B24044F9F7EF
:10E3300057F83088A188081830806D1CE8B2397908
:10E3400088420FD23868E9B201EB410200EB820447
:10E35000A088801CFF28CDD30C20BDE8F6810720C3
:10E36000BDE8F6810020BDE8F6812DE9FC4717469F
:10E370000546B7F80080002405F12C090E463C80C4
:10E3800099F8011071B3B8F1090FC0F0FD8068462B
:10E390006DDF002840F0F4803888082131541B21BB
:10E3A0003888401C3880062280B231540DF10101BA
:10E3B0003888401C388080B23044F9F711F8398829
:10E3C000891D39809DF80000400805D189B2745438
:10E3D0003888401C388005E089B20122725439889F
:10E3E000491C3980A878F8B13988091D8845C0F0E2
:10E3F000CB80684679DF002840F0C280398803204E
:10E40000705419213888401C388080B231543888C3
:10E41000401C388080B23044BDF800100170090AF9
:10E4200041703888801C3880E878A8B13988CB1CC6
:10E43000984540B2C0F0A880022272540122398867
:10E44000491C398089B272543988491C398089B293
:10E4500070543888401C38806868A8B139880057E3
:10E46000CB1C9845C0F09080022272540A22398851
:10E47000491C398089B272543988491C398089B263
:10E4800070543888401C3880288958B1CDF80480F1
:10E49000009733460622022105F10800FFF7C7FE68
:10E4A00004006ED1288A58B1CDF804800097334615
:10E4B0000722032105F11000FFF7B9FE040060D127
:10E4C000288B58B1CDF804800097334615221421CB
:10E4D00005F11800FFF7ABFE040052D1286A30B1F5
:10E4E00043463A463146FFF7B9FE040049D1D5F814
:10E4F00024A0BAF1000F30D0BAF804003988801C8B
:10E5000043189B1C98453FD3FF283DD2401C7054B4
:10E51000FF213888401C388080B231543888401C34
:10E52000388080B23044BAF800100170090A417096
:10E530003888801C3880BAF804206AB1DAF80810EC
:10E5400009B907241DE080B23044F8F749FF398843
:10E55000BAF8040041183980002499F8000038B155
:10E5600043463A4631462846FFF7BAFE040008D132
:10E57000287830B143463A4631462846FFF7B5FD84
:10E5800004462046BDE8F6870C24FAE738B4002894
:10E5900018BF002A22D00024651C8D4210DA15888D
:10E5A000AC4203DB05196D789D4209D02546045D18
:10E5B0002C19641CA4B2EFE7138080B232BC704700
:10E5C0008C420BDA005DA31C00281EBF401E84B2E3
:10E5D000002C03D014FA83F4A142EDDA32BC0020FF
:10E5E00070471CB504460020ADF8000013466A468B
:10E5F0002046FFF7CBFF10B1BDF80000204416BD48
:10E6000001F0C8B901F0D3B905E00A684B689A4235
:10E6100009D1083141600268416853689942F4D1D8
:10E62000002181607047826070470160096804E0E2
:10E630000A684B689A4207D1083141600268416814
:10E6400053689942F4D1002282607047816859B1C1
:10E6500003689A685118426881605368994203D1EF
:10E6600002F108014160CFE77047FEE730B4EFF3F5
:10E67000108272B6144B996871B901249C601349D9
:10E68000134C25680D401D602160616859604FF092
:10E69000FF316160002100E00121017002B962B622
:10E6A00030BC7047084A916861B158B9EFF31080E7
:10E6B00072B6084913680B6053684B600021916083
:10E6C00000B962B670470000CC6B0020FC06FFBDAD
:10E6D00080E100E000E100E0002818BF002901D13E
:10E6E0000E20704701601146026813681847F8B59C
:10E6F0000600154618BF002D0F461C4601D10E20FE
:10E70000F2BD306808B90820F2BD0CB90920F2BD8D
:10E7100017F0030F04D12246304600F089F808B9FB
:10E720001020F2BD234634682A46A5683946304693
:10E73000A847F2BDF8B50400154618BF002D0F46D6
:10E740001E4601D10E20F2BD206808B90820F2BD96
:10E7500036B160684068B6FBF0F100FB116008B1AB
:10E760000920F2BD17F0030F08BF15F0030005D113
:10E7700032463946204600F05BF808B91020F2BD59
:10E78000069800902A4620462468E56833463946B4
:10E79000A847F2BDF8B505000E4614461F4601D144
:10E7A0000E20F2BD286808B90820F2BD0CB9092076
:10E7B000F2BD68680268511E0E4205D162433146BF
:10E7C000284600F035F808B91020F2BD22462C6822
:10E7D000284625693B463146A847F2BD38B5002892
:10E7E0001CBF0168002915D10D490E480E4B091AAE
:10E7F000A1FB0332140909D00C4D296819B1C9696C
:10E800002846884720B91435641EF6D1002032BD51
:10E81000012032BDC969BDE834400847000000004E
:10E82000804400206C440020CDCCCCCC6C44002033
:10E83000C368994207D300695118491E8842804134
:10E84000C043C00F70470020704781680EE08168A8
:10E850000268491C914228BF002181600020704756
:10E86000C1688268914201D10020704700EB8100AD
:10E8700000697047C1680268491C914228BF0021A5
:10E88000C16000207047FEE71CB5049C0094001D89
:10E8900000F0BFFA16BD78B585B004460B208DF8A0
:10E8A00004000120224E234D31780090012301AA5B
:10E8B0002846FFF7E9FF30B931780C2302AA281D5A
:10E8C00000F0C0FA38B17188491C7180FCF75AFD1C
:10E8D0004FF0FF3028E002A89DF80810427842EA85
:10E8E0000122228081789DF80B2042EA01225242C7
:10E8F000628001799DF80D2042EA01225242A280F5
:10E9000081799DF80F2042EA0122E280017A9DF888
:10E91000112042EA012252422281817AC07A40EAE1
:10E92000012040426081002006B070BD0000000060
:10E9300068440020044300200000000000000000A4
:10E9400028B100BF22A1800141F0010108477047B2
:10E9500038B51B4D04462868B0F5967F2FD3A97DA6
:10E9600001292CD00120A875022000F0BBFDE87D14
:10E97000B0B94FF4FA71032000F064F8FEF704F91F
:10E98000FEF707F940F2A460FFF7DAFFFEF703F99C
:10E990004FF44870FFF7D4FFFEF702F9052000E0BE
:10E9A0000720FCF7B5FC0820FCF7B2FC2046FBF77B
:10E9B0004CF820462864BDE8324001F048B831BD2B
:10E9C000984200200000000000000000000000004D
:10E9D0000338FDD87047000010B52149214C0A6862
:10E9E00000E00C34A06840B120688242F9D3A068EE
:10E9F00080472168606841182160002010BD2DE922
:10EA0000F041194D2888D0B100242F1DA046144E86
:10EA10002888804510DA386808B9641C08E0316835
:10EA2000814205D3B868804700285CBF0020386069
:10EA30000C3708F10108EBE70CB900202880002012
:10EA4000BDE8F08110B5064C074B226889180C22EE
:10EA500050431844416005211980002010BD00007A
:10EA600098420020284300206443002001460320F0
:10EA7000CA0748BF4FF402408A0748BF48F2012046
:10EA8000490748BF48F202207047000001F12C03FB
:10EA9000D1F828C09A68624504D2496A895CC0F8F6
:10EAA0001C150FE01A7812B10121C16106E091F83E
:10EAB00020104A0604D50122C2615A700020704716
:10EAC0000121416101207047F8B400F582760022EF
:10EAD000336823B13260326800920122009B01F159
:10EAE0002C05EB787BB100243462336A0093002359
:10EAF000009CB361B36900930023009C736073684A
:10EB00000093009C25E0336AB3BBB469002C3CD170
:10EB10007368F3B1746073680093009C336A5BBBE5
:10EB2000AB688C6AA34214D200F5A064A6694C6A53
:10EB3000E654AB685B1CAB608C6A661EB34247D17F
:10EB400091F82060770643D40223C0F800320123F5
:10EB50000362002A4AD000226A70EA78002A42D171
:10EB6000AB68896A8B423CD000F5A060002101604F
:10EB700005210160012035E000233362336A0093F0
:10EB80000123009C4361EB70E3E7B361B369009339
:10EB9000009CAC68641CAC60336A002BECD18E6ABC
:10EBA000B44205D24B6A1B5D00F5A064E361D0E777
:10EBB0002B7813B10121C16115E091F820305C067A
:10EBC00003D50121C16169700DE001234361C0E7F4
:10EBD000A342BCD10B6A5C06BBD5B8D502206870D5
:10EBE00001E00020E870F2BC00207047F2BC012078
:10EBF0007047FEB50446DFF83C030090002504F59D
:10EC000082700E46056006F12D0701680191019A98
:10EC10000562016A0191019A856181690191019AF8
:10EC200045604068019001200199C4F80052756365
:10EC3000BD702062387801281CBF0121A1603146D7
:10EC40002046FFF723FF3068E8B140F28621B1602B
:10EC5000B068C4F8040315E031462046FFF734FFDE
:10EC600000281EBF0098401E00900CD10EE0032526
:10EC70000098012806DA04F2C4400021C16303258C
:10EC80000521C1636DE000990129E5DAB878002813
:10EC9000EED004F2C441086808600028E7D0FFF70E
:10ECA000E5FE0546E4E7FEB50446A24800900025CF
:10ECB00004F582700E46056006F12D07016801918A
:10ECC000019A0562016A0191019A85618169019148
:10ECD000019A45604068019001997563BD70B06A02
:10ECE000012805D196F82010480658BF022000D50B
:10ECF0000120C4F80002012020623978022918BFDF
:10ED000020603068E8B140F28621B160B068C4F894
:10ED1000040315E031462046FFF7D6FE00281EBF4B
:10ED20000098401E00900CD10EE0032500980128A9
:10ED300006DA04F2C4400021C16303250521C16342
:10ED40000FE000990129E5DAB8780028EED004F246
:10ED5000C441086808600028E7D0FFF787FE054631
:10ED6000E4E7284603B0F0BD2DE9FC410D4605F16E
:10ED70002C04617801290DD1117801290FD000F5FB
:10ED800041766B4F7760217961B1A86830601120BE
:10ED9000BDE8F6810229F2D111780129EFD00820CF
:10EDA000BDE8F6819E0806F0010686F00106267190
:10EDB0002B6205F10C0192E8C05181E8C051516805
:10EDC000A962D16869625178C0F888151178012963
:10EDD0000AD0002906BF5B0903F001030123237059
:10EDE0002946FFF706FF02E02946FFF75CFF296886
:10EDF00009B900222271BDE8F68130B413460479C6
:10EE000000680A464949C4EB041501EB850130BC92
:10EE1000AAE7F0B585B06D460A9C00260027B446E7
:10EE2000A5E8C010C0C58DF8011003920193002C15
:10EE300014BF202200226946FFF7DFFF05B0F0BDB6
:10EE4000000000002DE9F8413DA595E8C05185B0CE
:10EE50006C4684E8C0518DF80110039201930022A2
:10EE60006946FFF7CAFF06B0BDE8F081F8B586B085
:10EE700005460C46FFF728FE00284DD104F12C0171
:10EE8000C878F0B9207B022811BF0328626AA36901
:10EE90009A4216D1E269626200236269A262226A22
:10EEA0004B70520902F001020A70032821462846DD
:10EEB00003D1FFF79EFE07B0F0BDFFF7F4FE07B0E9
:10EEC000F0BD04F10C0292E8C85001A880E8C850D7
:10EED000C87898B1D5F8C404C5F8C404820748BFFF
:10EEE00001200BD4420748BF022007D4C20748BF05
:10EEF000032003D404228DF8002001E08DF80000E7
:10EF000000220A7194F82000420701D5C87818B190
:10EF1000616822686846904707B0F0BD034906481B
:10EF2000A4E706494FF04020A0E70000DC6800207D
:10EF300086420400A08601000030004018690020CD
:10EF400001000000000000000000000000000000C0
:10EF50000000000011B581B000218DF80010684656
:10EF6000FFF784FBFDF77EF850B9424C01A920461B
:10EF700000F090FD204600F07FFD08B100F079FE22
:10EF80009DF80000FFF78EFB13BD000038B53A4D29
:10EF90002978002409B1852032BD00B938A0008845
:10EFA000A5F801008DF800406846FFF75FFBFDF70C
:10EFB00059F838B93149681C00F02AFE040008D11C
:10EFC00000F049FE012028709DF80000FFF76AFB61
:10EFD000204632BD2DE9F84605468946002742F213
:10EFE0000706DFF890A000218DF800106846FFF7B3
:10EFF0003DFBFDF737F8040007D14A462946504645
:10F0000000F0E6FD074600F026FE9DF80000FFF741
:10F0100049FB2CB14946284631DF0746B74204D0A8
:10F02000022FE0D03846BDE8F2860527FAE780B522
:10F0300010B1032809D001BD0F480178012918D16A
:10F0400000F017FE00F01BFE01BD00208DF800004F
:10F050006846FFF70BFB08480178012905D10749ED
:10F06000401C00F0D5FD00F0F6FD9DF80000FFF714
:10F0700019FB01BD480C0300446C002055EF020051
:10F080000106FEE70268012111600223FFE7007913
:10F09000394900EB400201EB82010B7270470068B6
:10F0A00001210160704700680121416070470068DC
:10F0B0000121C160704778B400684FF480348C40FF
:10F0C00000F5417553B14FF4A07303EB81030026A3
:10F0D000C650C3580093009E2C6000E06C6000EBAB
:10F0E0008100C0F8402571BC7047FCB41C4605681F
:10F0F000069BD5F8006240F201178F40BE43C5F869
:10F100000062D5F800623443C5F8004202B0F0BC9A
:10F11000D1E72DE9FC410546904600275FEA08004B
:10F120000E461BD04FF480344FF4A07000EB8702E2
:10F1300011B2685800281EBFD5F8043304FA07F04E
:10F14000034208D0002068506858009010B200991F
:10F150007168326890477F1C4745E5DBBDE8F38165
:10F16000042205490548D4E7042205490548D0E7AB
:10F17000042205490548CCE7D06A00200080004001
:10F18000DC6A002000900040E86A002000A00040F7
:10F190000F480168084738B50D460E49884214D11A
:10F1A00000248DF800406846FFF760FA08490879A6
:10F1B000002811BF01240D6001220A719DF8000092
:10F1C000FFF770FA0CB1112032BD002032BD0000F3
:10F1D000186C002000200040034600E05B1C1A78F9
:10F1E000002AFBD111F801CB83F800C013F801CB42
:10F1F000BCF1000FF6D170471CB50446F8F792F841
:10F20000204410F8021D0D2918BF0A2902D100213F
:10F21000017013BD41780D2912BF0A2900214170E8
:10F2200013BD0246C9B2002013788B4208BF1046B6
:10F2300012F8013B002BF7D17047000000000000DE
:10F2400010B5040008D00FF2A8314FF47A4041F015
:10F2500001018847641EF6D110BD0000F8B50026F4
:10F26000012840F2EF1540D10A240FF20437FDF7D0
:10F2700084FC00F0DDF8FDF782FC00F0D9F800F026
:10F28000D3F8FDF77AFC00F0D3F8FDF778FC00F036
:10F29000CFF800F0C9F8FDF770FC00F0C7F8FDF7F3
:10F2A0006EFC00F0C3F8FDF768FC00F0BFF8FDF756
:10F2B00066FC00F0BBF8FDF760FC00F0B7F8FDF766
:10F2C0005EFC00F0B3F8FDF758FC00F0AFF8FDF776
:10F2D00056FC00F0ABF800F0A4F800F09DF800F048
:10F2E00097F8761C641EC2D1F1BD02283FD10A24D2
:10F2F000A8A7FDF742FC00F09BF8FDF740FC00F0EA
:10F3000097F800F091F8FDF738FC00F091F8FDF760
:10F3100036FC00F08DF800F087F8FDF727FC00F0D0
:10F3200085F8FDF725FC00F081F8FDF726FC00F0DC
:10F330007DF8FDF724FC00F079F8FDF717FC00F0EC
:10F3400075F8FDF715FC00F071F8FDF716FC00F0FC
:10F350006DF8FDF714FC00F069F800F062F800F0B9
:10F360005BF800F055F8761C641EC2D1F1BD00BFF9
:10F3700091A70A24FDF701FC00F05AF8FDF7FFFB06
:10F3800000F056F800F050F8FDF7F7FB00F050F8E9
:10F39000FDF7F5FB00F04CF800F046F8FDF7EDFB4B
:10F3A000FDF7E4FB00F042F8FDF7E9FBFDF7E0FBB9
:10F3B00000F03CF8FDF7E1FBFDF7D8FB00F036F874
:10F3C000FDF7DDFBFDF7D4FB00F030F8FDF7D5FBD2
:10F3D000FDF7CCFB00F02AF8FDF7D1FBFDF7C8FBE9
:10F3E00000F024F8FDF7C9FBFDF7C0FB00F01EF8A4
:10F3F000FDF7C5FBFDF7BCFB00F018F800F011F8B5
:10F4000000F00AF800F004F8761C641EB2D1F1BDD9
:10F4100031463846F9F7B9BC324639460120F9F78A
:10F4200057BF4FF4FA600BE7284609E7FA2007E7D1
:10F43000642005E780B53DE080B54DE03E480168B9
:10F44000491C0160C80748BFFDF797BBFDF78EBB9D
:10F4500039480178CA0748BFFDF791BBFDF788BB63
:10F4600035480168491C01600320B1FBF0F000EB56
:10F470004000091A012908BFFDF77FBB70472E48DD
:10F4800000680321B0FBF1F101EB4101401A0128B2
:10F4900008BFFDF774BB704727480168491C01602D
:10F4A0000320B1FBF0F000EB4000091A012900D065
:10F4B000704780B5FDF761FBBDE80140FDF756BB25
:10F4C0001D4800680321B0FBF1F101EB4101401A36
:10F4D000012800D0704780B5FDF751FBBDE8014021
:10F4E000FDF746BB10B50446FDF749FBFDF740FBB1
:10F4F000012C20461149124A18D0022C02D1114980
:10F50000114A13E0032C02D11049114A0EE0042CD9
:10F5100002D11049104A09E0052C02D10F49104AC6
:10F5200004E0062C06BF0F490F4A01200F4B9A60DA
:10F530005960186010BD0000406C00206DCB0200C7
:10F5400071CB02007BCB02007FCB020035F40200BE
:10F5500039F402003DF4020051F4020061F40200AB
:10F560007FF4020099F40200C1F402007C42002002
:10F57000494D552073656E736F722C206E6F742029
:10F58000646574656374656421212120633D25648D
:10F590000D0A00004163747561746F722C206E6FE8
:10F5A0007420646574656374656421212120633D62
:10F5B00025640D0A0000000045787465726E616C68
:10F5C000206D656D6F7279206973206E6F74204FA6
:10F5D0004B21212120633D25640D0A00000000001D
:10F5E000000000000000000000000000000000001B
:10F5F0000338FDD87047000004E010F8013B6BB100
:10F60000491C521E52B10B7890F800C09C45F4D0B2
:10F6100002D24FF0FF307047012070470020704742
:10F6200033B58BB00446002000900C9981B10025C1
:10F6300029460CA800F06FFB38B10098694601EB31
:10F64000400295800098401C00906D1C142DEFD353
:10F650002046694687E082B012B102B000F046BB96
:10F6600002B000F04DBB2DE9F04F074697B0388847
:10F67000B7F80480102806D0112845D0192865D085
:10F680001A2846D06CE0DFF80461B068C0430090EF
:10F690006846716800F056FB00990CA8FFF7C0FFA0
:10F6A00001A80CA92C22F7F7ABFE019898B10DF137
:10F6B00008090546B9F800A006F1040B1E245146BE
:10F6C000584600F01DFB641E0BF1040BF7D16D1EB4
:10F6D00009F10209EED1B8F1140F03DB0420FBF7A6
:10F6E00091FE3DE0414606F1080000F0FFFA414678
:10F6F000301D00F0FBFAF87B022831D1414606F1BB
:10F700000C0000F0F3FA2BE04146214800F0F8FA33
:10F7100026E03D7A1D4C2D09042DACBF01220022AC
:10F72000414604F11800FFF796FF022DCCBF0122DD
:10F730000022414604F11400FFF78DFF022DACBFFB
:10F7400001220022414604F1100007E0387A38B95E
:10F750007A7A1048D20802F001024146FFF77BFF97
:10F7600017B0BDE8F08F2C22F7F74AFE0DB030BD80
:10F7700010B51428044606DA2146074800F0CBFAF3
:10F7800008B1204610BD142010BD000060680020A4
:10F79000686800207868002064680020000000008D
:10F7A0000068D0F80405704790F90410080007D4E9
:10F7B000012201F01F00064B8240490943F8212035
:10F7C000704702490868896808470000FC6B002000
:10F7D00000E200E0000000000000000050B411B999
:10F7E00050BC0E207047144694FBF3F603FB1644FE
:10F7F00014B150BC09207047016082810021416032
:10F800008160C381002050BC7047000081B050E887
:10F81000022FC188B2EB324F4FF0000317BF92B2F4
:10F8200041EA014142EA014104E04268B2EB324F51
:10F8300008BF012340E80212002AE8D18DF8003009
:10F840009DF80000002814BF0020112001B070476F
:10F850003CB450E8015FAAB2C3891A4483899A4232
:10F8600028BFD21A03899A4202BFBFF32F8F002408
:10F8700007E0C2EA050240E80123002BE9D14FF07E
:10F88000010401958DF80040019A0A609DF800205E
:10F89000002A1DBF006809884018002036BC704748
:10F8A0000A8849888A4209D150E8011FC1EA01410A
:10F8B00040E80112002AF7D101207047002070476C
:10F8C0003CB450E8025F1FFAA5F2C3889A4202BF17
:10F8D000BFF32F8F00240DE0C3891A4483899A4215
:10F8E00028BFD21AC5EA024240E80223002BE8D121
:10F8F0004FF0010401958DF80040019A0A609DF8CF
:10F900000020002A1DBF006849884018002036BC2E
:10F91000704700000A8849888A4209D150E8021FCE
:10F92000C1EA214140E80212002AF7D101207047C4
:10F9300000207047401810F0030308D0C91A1FD3E5
:10F94000DB0748BF00F8012D28BF20F8022D130067
:10F9500030B414461546103928BF20E93C00FAD8C7
:10F96000490728BF20E90C0048BF40F8042D890052
:10F9700028BF20F8022D48BF00F8012D30BC704789
:10F98000C91818BF00F8012DCB0728BF00F8012DBA
:10F990007047FEE780B51548002141700161BFF353
:10F9A0005F8F001D13A1FEF740FE002002BD80B551
:10F9B00000218DF800106846FEF758FEF1EE100A9F
:10F9C00020F09F00E1EE100ABFF35F8F084840214E
:10F9D00001609DF80000FEF765FEFCF743FB08B1EF
:10F9E00041DF01BD20BF40BF20BF01BDA86B00208B
:10F9F00084E200E0180C0300300C03000400000057
:10FA000080B5012289B2F9F716FC05490A68002879
:10FA100004D4521CB2F57A7F28BF00220A6002BDCE
:10FA2000286C002000B5A1B08023009301AB00F04A
:10FA3000A5F901460129B2BF4FF0FF3001A8FFF739
:10FA4000DFFF21B000BD002200210120EAE70146CE
:10FA500000220020E6E7024604210520E2E70146F5
:10FA60000A6810685268824201D3101A7047896888
:10FA7000491C081A1018704702681168526880689B
:10FA8000824234BF521C00228A4201D101207047B9
:10FA900000207047F8B5044600250E468DF800504A
:10FAA0006846FEF7E3FD2046FFF7E6FF00281CBF8F
:10FAB000217C002941D121684B684A68A768BA4275
:10FAC00034BF521C00224A6030B10868A2689042DC
:10FAD00034BF401C00200860E268012A06D0022AD8
:10FAE00008D0042A0BD0082A0ED015E061683078BF
:10FAF000C85418E06168308821F8130013E0616889
:10FB0000306841F823000EE06268D6E9000102EB9C
:10FB1000C302C2E9000106E0606802FB030331464C
:10FB20001846F7F75DFC2046FFF799FF21688B68C0
:10FB3000984238BF1846886000E004259DF8000010
:10FB4000FEF7B0FD2846F2BD0246136818685B68F0
:10FB500039B1834203D39168491CC81A7047C01A4F
:10FB60007047834201D3181A70479268521C101ACA
:10FB700070472DE9F843044688462068D0F8009085
:10FB8000154600212046FFF7DFFF0646E76861685B
:10FB9000AE4207FB09110AD307FB05F24046F7F70F
:10FBA0001FFCA0684D44A8420ED200250CE077430C
:10FBB0003A464046F7F714FCE2686168AD1B6A43B9
:10FBC00007EB0800F7F70CFC20680560BDE8F1833F
:10FBD000F8B505460E46144600270CB90020F2BDC4
:10FBE0008DF800706846FEF741FD2846FFF737FFA5
:10FBF000A04205D3224631462846FFF7BAFF00E06F
:10FC000005279DF80000FEF74DFD3846F2BDFEE7E2
:10FC10002A4B1A780AB18520704759600178CA07C3
:10FC200004D527490A6842F001020A602549D1F843
:10FC300000C04FEA5C0C4FEA4C0CC1F800C04078A1
:10FC400021494001087021484FF400510160012012
:10FC50001870002070471E4881B0002101600068C4
:10FC60001C4A0090012000991B491060086001B0F7
:10FC700070471A491A4A01200860106070471749F6
:10FC8000174A0120086010604FF40050154A1060B8
:10FC9000BFF34F8FBFF36F8F0021084A1170704779
:10FCA0000B4882B0002101600068044A009000996E
:10FCB0000D4800685168C0B202B00847206C0020AF
:10FCC00004D5004000D200400DE400E000E100E077
:10FCD00000D1004004D3004000D0004008D30040D1
:10FCE00004D0004080E100E008D500400B4601212F
:10FCF00003F01F025B09914000EB830000F014B891
:10FD00000B46012103F01F0291405B09C94300EB40
:10FD1000830000F017B84A0950F8220001F01F01D3
:10FD2000C84000F00100704710B4024652E8004F8E
:10FD300044EA010042E8000393F0000FF6D110BC42
:10FD40007047000010B4024652E8004F04EA010078
:10FD500042E8000393F0000FF6D110BC704700009A
:10FD600010B40146012451E8000F40EA040341E8C1
:10FD7000003292F0000FF6D110BC70472DE9F84F19
:10FD800001288AB09846DFF8D890364F17D105A8D9
:10FD9000FAF700FFFCF749FC3968334A136803900F
:10FDA0000491019309F1190330480168029105A8F3
:10FDB0000090012231A14046FBF704FB4DE00028F2
:10FDC00018BF02280C4637D1002C0CBF4FF0000B97
:10FDD0004FF0020BFCF7F5FE0546FCF7F6FE05407A
:10FDE0000795FCF722FC3968214EDFF888A0224DE8
:10FDF000BAF80020069101237188521A05923188C1
:10FE00002A880290521A049209F11900079A039263
:10FE1000009001944FEA0B0220A14046FBF7D2FA72
:10FE200029883288914218BF3180BAF80010728850
:10FE3000914212D0718010E0052808BF042C0AD12D
:10FE400038680190009209F1190301221BA1404674
:10FE5000FBF7B8FA01E04FF0FF300BB0BDE8F08FD0
:10FE600098420020286C0020D44000203C6C0020E8
:10FE7000306C00206A6B00206A440020513D313B09
:10FE8000323B25643B25733B25732C25732C253091
:10FE900038582C25643B256400000000513D256442
:10FEA0003B323B25643B25733B25642C25642C2584
:10FEB000642C25642C25643B25640000513D353BB2
:10FEC000323B25643B25733B342C25643B25640081
:10FED000024613689868002800D1704770B586B054
:10FEE0006B4600240025002670C370C30191906802
:10FEF0000590107910B101280AD011E001208DF889
:10FF0000000011690291D06803905069049007E0E5
:10FF100002218DF80010D06800030290516904910D
:10FF2000684611688A68904706B070BD1CB59D4C44
:10FF3000217A49B904F1B40104F1A400FFF7C0FC2F
:10FF4000606108B9606013BD02206369207218798E
:10FF500010B1012813D024E098695A69121AB2F539
:10FF6000805F09D29208012A98BF0122D9681B69D3
:10FF70004118C01829DF06E04FF48062F6E7D86820
:10FF80001969081828DF10B1112807D009E0207C72
:10FF9000B0B9BDE81C40002102209FE00120207282
:10FFA00013BD60690321FFF793FF0020207260609A
:10FFB00004F1B40104F1A400BDE81C40FFF7AABCA1
:10FFC00013BD10B5774C201DFFF7CAFE002804BFF3
:10FFD000607C002802D1BDE81040A7E710BD0000FA
:10FFE00010B500BF71A16F4C41602046FFF7B8FE0D
:10FFF00050B9FCF737F820741C238C2204F1180147
:020000040003F7
:1000000004F1A400FFF7EAFB002010BD10B5654C19
:1000100014212046FAF74AFC04F1A400FFF7F6FB8E
:10002000002010BD2DE9FC4706460D46DFF878811B
:100030009246994669464046FFF70AFC040008BF0D
:10004000042013D00A9F1C21FEF74CF800202071D9
:100050002660A7602561C4F80CA0C4F81490694616
:100060004046FFF71DFCFFF7ACFF0020BDE8F68718
:1000700080B510461A46F7F7B3F9002002BD2DE906
:10008000F84381460F46DFF8208115461E46694633
:100090004046FFF7DDFB040008BF042011D01C21FF
:1000A000FEF720F801202071C4F80090A6603F0BF5
:1000B000E760656169464046FFF7F2FBFFF781FFA5
:1000C0000020BDE8F283084670470020704735489D
:1000D000017A481E8041C043C00F70471CB50228FA
:1000E00018BF032843D12F4C217A00293FD0022981
:1000F00034D1022802D003281ED02FE060690021ED
:10010000E160017959B1012928D10169491C0161D6
:100110004069814222D100202072002115E08169CE
:100120004269531AB3F5805F88BF4FF48053591862
:100130009142816112D1EEE7E068401C0928E0603D
:100140000CD30020E06020720D216069FFF7C0FE33
:1001500004F1B40104F1A400FFF7DCFB607C10B9EA
:10016000BDE81340E2E6BDE81340FBF770BF13BDE6
:100170000C4801214174007A401E8041C00F704735
:10018000012882B004D1074900204874012004E00E
:10019000032805D1034900204874087402B0C5E65D
:1001A00002B07047A86700204C68002000100000D3
:1001B000040000000100000000000000000000003A
:1001C00028B100BFAAA1800141F001010847704792
:1001D00010B5040005D04FF47A70FFF7F1FF641EEC
:1001E000F9D110BD80B573480068410508D50120DC
:1001F000FFF734F8BDE802400320FBF789B801BDE2
:10020000010448BF0220F3D4810448BF0320EFD487
:10021000C005F4D50420EBE71CB501226946012096
:10022000FAF7CCFB0028644C04D40098012804BFE2
:1002300001212176012269460220FAF7BFFB00283E
:1002400005D40098401F1A283CBF0098E06513BDF4
:1002500038B590B0FCF76CFC0028564C03D52068EC
:1002600040F001002060FCF788FCF8F75FFD0028F3
:1002700003D5206840F0040020601420FFF7A0FFA1
:10028000F9F72EFB002803D5206840F48040206059
:100290001420FFF79DFF00F0EFF84848D0F8001059
:1002A00047A0F8F772FD00BF4DA0F8F76EFDFEF70E
:1002B000A7F9FCF756F9002803D5206840F4007030
:1002C00020603D4D05F11900F9F706FA37A105F157
:1002D0001900F9F76FFB70B96846FAF776FC6B46C0
:1002E0005FF0010242A105F11900FBF76BF805F17F
:1002F0001900F9F7EFF96846FAF7C4FB6846F7F713
:1003000011F804281AD205F11900F7F70BF80C2898
:1003100004BF687E53280CD1A97E572904BFE87F0B
:10032000432806D105F1190234A16846FBF74AF8C3
:1003300004E005F119016846FAF7BCFA4FEA0D012D
:1003400032A0F8F722FD6846F8F742FF002803D5EF
:10035000206840F4803020601420FFF739FF00F05F
:100360008BF86846F8F7D6FF4FEA0D0205F1190140
:100370002AA0F8F70AFDFFF74FFF0DA0F8F705FDDB
:10038000FAF7BEFFFCF7FBFBFCF7F2FB206838B185
:10039000FFF728FF26A0F8F7F8FC4FF0FF3003E046
:1003A00028A0F8F7F2FC002011B030BD58585800D2
:1003B0000D0A00003C6C002098420020D440002030
:1003C0000D0A53746172742120434C4B3D36344DF9
:1003D000487A2C205665723D25730D0A0A000000EC
:1003E0003C5253542D42312E303E0D0A0A0000007B
:1003F00053572530326425730000000053575F4186
:100400004952424147202D2025730000424C455F50
:100410004E414D45203A2025730D0A000D0A4944EE
:10042000203A20257320282573290D0A0A00000090
:1004300053797374656D204661696C757265210D21
:100440000A0A000053797374656D205265616479FE
:10045000210D0A0A0000000000000000000000005A
:10046000000000000000000000000000000000008C
:100470000338FDD87047000080B500F0B1F818B11E
:10048000FAF780FF4FF0FF3002BD000078B5DFF8CB
:100490007061DFF8705183B0706805F12D0420B3EE
:1004A00000217160706800900099607808B1A178AF
:1004B000D9B16968019100228DF800202989ADF831
:1004C0000810E96809B92A740AE02A8B6A8369600E
:1004D0002A810021E96018B9DFF82C0101210160AF
:1004E00068462A6890470020A070617800291CBFE8
:1004F000306800282DD000213160316800910098CB
:1005000021786A8B91420AD2501A688380B22B8973
:100510006C68DFF8F820181A04EB400009E08A4202
:100520000ED1E86840B10122A27000226A83DFF890
:10053000DC201060516003E00120A070002068837F
:1005400000207060DFF8C0207068009001200099E2
:100550005060306960B10021316130690090002045
:100560000099287402208DF80000684629688847A1
:10057000706918B96C694FF000462DE00020706179
:100580007069009000200099287404B070BDB4FA1E
:1005900084F026FA00F18C43810001F58C7109B2D8
:1005A000DFF864205058B8B100235350A1F58C7384
:1005B000525800920906890E01F0010181F00101F3
:1005C00000988DF805100122DB088DF800208DF8C9
:1005D0000430684629688847002CD8D104B070BD23
:1005E0000B490A780020012A01D008207047897F32
:1005F000054A11B10123136070470123536070470E
:1006000000710040486A0020007000402C760040D5
:10061000586A0020BFF34F8F7E497F480A6802F472
:10062000E06202430A60BFF34F8F00BFFDE7F8B5F9
:100630007E487F4A016811F1010F08BF1178062931
:1006400005D17C490B68C3F304217B4B19601378F7
:10065000062B02BF9168C1F30311032902D1774B26
:100660007749196003687749774C13F1010F08BF88
:100670001378062B03D12368C3F342334B601578FC
:10068000724B062D02BF9568C5F30315032D03D1E8
:100690005D6F25F080755D67056815F1010F08BF76
:1006A0001578062D04D16A4D00262E606E600E600E
:1006B0001578062D01BF9568C5F30315032D8D66CA
:1006C0001578062D02BF9568C5F30315032D08D1D3
:1006D000604D05262E600126AE670026AE603F26DF
:1006E0006E60056815F1010F03BF15789668C6F3B3
:1006F00003164668062D26D1F61E012E23D9564E26
:10070000564D37682F6077686F60B768AF60F768DD
:10071000EF6037692F6177696F61B7692F62F76999
:100720006F62376AAF62776AEF62B76A2F63F76A00
:100730006F63376B2F64776B6F64B76BAF64F76B66
:10074000EF64366C2E65056815F1010F08BF15784A
:10075000062D04D16469424D04F04F042C600468F6
:1007600014F1010F08BF1478062C06D13D4A146815
:10077000E50744BF6FF0010515600268062A08D13D
:100780004468E41E022C04D9374A146844F4806497
:1007900014601A6842F470021A60BFF34F8FBFF3FF
:1007A0006F8F0368314A062B05D14068C01E0328AD
:1007B00084BF90680862D068194B184CC10709D5EE
:1007C0000121216018680028FCD0D5686D086D00F3
:1007D000D56011E0116800295CBF5068002815D56C
:1007E0000121216019680029FCD0152010601868CB
:1007F0000028FCD01521516019680029FCD0002088
:10080000206018680028FCD0FFF704FF054806495F
:100810000160F1BD0CED00E00400FA0504E50140C3
:1008200000E40140244300200090D0033001001078
:10083000E00F00F0240300104035014074C0074071
:100840000DF0ADBA380500404402001088ED00E01C
:100850000C010040105600400404001020C5004068
:10086000E40E0040000400403C170040001200105D
:1008700080B500BF20A0F8F788FA1C4A012182F851
:100880000411FFF7E0F8002804D40020FFF7DFF898
:10089000002002BD4FF0FF3002BD80B50320FAF703
:1008A00037FD002002BD80B511480168B1F5967F83
:1008B00000D2EFE70420FEF715FE0E490220088063
:1008C000002002BD80B5FCF771F9002002BD0000D8
:1008D00080B507480021C175D0F800100FA0F8F7C7
:1008E00054FA0020FFF7B7F8002002BD8044002032
:1008F000984200206443002072756E5F6F6E6365DE
:100900005F6F6E5F636F6E6E65637465645F686171
:100910006E646C657228290D0A0000002564202091
:10092000747269676765722C20656E61626C6564BC
:100930002E0D0A0010B5FFF79FFDFBF773FE224C4A
:10094000617D40F2C67290420DD209B901206075F6
:10095000206910B90620FEF7C5FD206906281FD2C0
:10096000401C20611CE0A0F2C77039280ED2B9B932
:10097000206900B12161E068401C0128E0600FD9C6
:10098000012060750520FEF7ADFD09E0012907D1C2
:10099000002060750120FEF7A5FD00202061E060C9
:1009A000002010BD80B5094801688847002002BDBD
:1009B00080B5074908688047064A108808B1FEF7E5
:1009C0001EF8002002BD0000984200208042002056
:1009D000844200206443002080B50020FFF737F8F0
:1009E000002002BD7365740073686F77000000001B
:1009F00064667500646E74006578636C65616E0092
:100A0000636C65616E00000064756D70000000002D
:100A10007265736574000000737461727400000085
:100A2000656E61626C65000064697361626C65008B
:100A3000777269746500000068656C7000000000E2
:100A4000636C6F73650000001FB500BF0CA40EE05F
:100A5000052818BFFAF7D6FC1FBD51680098126828
:100A6000904701A8FDF7F2FD039A002AF5D16846E8
:100A70004BDF0028ECD1214601A8FDF7D6FDF3E7B6
:100A80006C0C03007C0C03000800000019E050F817
:100A9000042BD30744BFA9F101039A18091F0023AF
:100AA000042942F8043BF9D25FEA817C134604D55D
:100AB0004FF0000CA2F800C09B1CC90744BF0021E6
:100AC000197050F8041B0029E1D17047E80C0300AD
:100AD000F00C03000000000000000000AC0C03005C
:100AE000BC0C030000000000000000009C0C030090
:100AF000AC0C03000000000000000000000000003B
:100B000038B500BF06A5642445F001054FF47A40CE
:100B1000A847641EFAD1FFF79BFBFBF769F9FCE7D6
:100B20000338FDD87047000010B5074979441831E3
:100B3000064C7C44163404E00A68081D11448847BA
:100B40000146A142F8D110BD2C0000005800000061
:100B50004EF68851CEF20001086840F4700008603B
:100B6000BFF34F8FBFF36F8F4FF00070E1EE100AAD
:100B70007047000019FFFFFFD827000080440020C5
:100B8000000000001366FFFF90010000F402000067
:100B9000004000200366FFFFFA0200002200000070
:100BA0006C440020FEE70000D80C0300E00C0300BA
:100BB000300C0300480C03008C0C03009C0C030059
:100BC000E00C0300E80C0300E1FF02000D0003004D
:100BD00071000300250003007F000300C70003002D
:100BE000CB000300CF0003000120C046002801D045
:100BF000FFF79AFFAFF300800020AFF30080FFF70C
:100C00007FFF00F000F800F001B8FEE70746384625
:100C1000F7F7CAF9FBE7FEE700000000000000005C
:100C200000000000000000000000000000000000C4
:100C300089C20200946B002055BD02008845002047
:100C40001BB9020000000000D86B0020C46900201E
:100C500040000000010000000000000042582D4E3E
:100C600052462D312E352E3100000000F00C0300CD
:100C7000F80C03000000000000000000014880475D
:100C8000014800472F060300BD0C0300B5B5020064
:100C9000F040002081B402000C41002099C1020004
:100CA00000000000490A0300000000008101030069
:100CB000000000002FF0020000000000AFF30080F1
:100CC000FFF746FFFFF790FF000000000000000064
:100CD0000338FDD87047000067F6020000000000EE
:100CE000AF9002000000000071010300000000004E
:100CF000DD0003000000000000002E004300FEE7BE
:100D0000FEE7FEE7FEE7FEE7FEE7FEE7FEE7FEE7BB
:100D1000FEE7FEE7FEE7FEE7F20B0001F0055710E5
:100D20000140110004000110021F1C1F1E0241059A
:100D3000821D0CF11B8112FF01100B5C0C0300FCE7
:100D4000080000346C002001C0F0010CFFFF1443C8
:100D5000E002DC40002021F0058001000200534445
:100D600000013001E4090395100369830200E80CD7
:100D700050070101000063850200F00C1005A580FA
:100D80000200248902C010010000750C52F41812F0
:100D9000ED0C222C18110C5003A7810200F818400A
:100DA000046D820200000A0C12095452080C500310
:100DB0008D860200100C12910C52180C12B90C43C3
:100DC000200A8412C30C52280C50032587020030DD
:100DD0000C127B0C52383012BD0C52401812B30C5E
:100DE000210121182101210710036DCB020071049C
:100DF000311AF4013330024072F2120145E20A2442
:100E00007330007C3140700140004048100290D0A7
:100E1000031B0C1403B80B00003538122F0C12649E
:100E20000412A50C52390C12B10C124308B0057013
:100E3000170000D909035E92050E8371081C129BEE
:100E40000C699A92A71892C50C12D10C8001053535
:100E500015425220A8F71C20002CF00108F80C03C2
:100E60000452FF01F200FA1410010000FC0C2508E6
:100E7000FF01E8432403210110031D720200110445
:100E800070013172021F52D90C7401C772028C12A8
:100E90006808520001000A61C5020000800600FFD8
:030EA0009F0600AA
:0400000500030CBD2B
:00000001FF
